:10142400758400852ED2852FD37584018530D285AD
:1014340031D3E4F52FF52E30005730064E855B820C
:10144400855A83E0F52FA3E0F52EA385825B85837F
:101454005AE55B655D700CE55A655C7006755B006A
:10146400755A02855982855883E533F0A3E532F035
:10147400A3858259858358E559655D7014E55865DF
:101484005C700E755900755802800685322E8533BE
:101494002F30010CE52E2534F52EE52F3535F52FAB
:1014A400300210E53F8527F0A4252EF52EE5F03512
:1014B4002FF52F300310E50A852AF0A4252EF52EEA
:1014C400E5F0352FF52F300410E5118529F0A4251A
:1014D4002EF52EE5F0352FF52FE4F531F5303009F2
:1014E4005730054E855B82855A83E0F531A3E0F5DC
:1014F40030A385825B85835AE55B655D700CE55A94
:10150400655C7006755B00755A028559828558833F
:10151400E535F0A3E534F0A3858259858358E55970
:10152400655D7014E558655C700E75590075580258
:10153400800685343085353130080CE5302532F5A8
:1015440030E5313533F531300A10E53F8527F0A415
:101554002530F530E5F03531F531E531C3952C40D2
:0315640003852CD0
:1015670031300B10E50A852AF0A42530F530E5F077
:101577003531F531300C10E5118529F0A42530F50A
:1015870030E5F03531F531300D10E5188528F0A438
:101597002530F530E5F03531F531E531C3952D408E
:1015A70003852D31229016053015031215C230160A
:1015B700031215D23018031215F522E50B2509F58C
:1015C7000BE50C3508F50C93F50A22E512250EF507
:1015D70012E513350DF51393C313F8E5142510F52C
:1015E70014E515350FF51593C31328F51122E519E1
:1015F7002517F519E51A3516F51A93F518227F827E
:1016070085888C8F9295989B9EA1A4A7AAADB0B30D
:10161700B6B9BBBEC1C3C6C9CBCED0D3D5D7D9DC2B
:10162700DEE0E2E4E6E7E9EBEDEEF0F1F2F4F5F601
:10163700F7F8F9FAFBFCFCFDFDFEFEFEFEFEFEFEE2
:10164700FEFEFEFDFDFCFCFBFAFAF9F8F7F6F4F3F3
:10165700F2F0EFEDECEAE8E7E5E3E1DFDDDBD8D632
:10166700D4D1CFCDCAC8C5C2C0BDBAB7B4B2AFAC6A
:10167700A9A6A3A09D9A9794908D8A8784817E7A44
:101687007774716E6B6865625F5C595653504D4A4B
:101697004744423F3C393734322F2D2A282624210C
:1016A7001F1D1B1918161412110F0E0C0B0A080711
:1016B7000605040403020201010000000000000007
:1016C70000000001010202030405060708090A0BCE
:1016D7000D0E1011131516181A1C1E202224272967
:1016E7002B2E303335383A3D404245484B4E515406
:1016F70056595C606366696C6F7275787B7FFEFE16
:10170700FEFEFDFCFCFBFAF8F7F6F4F3F1EFEDEB68
:10171700E9E7E4E2DFDCDAD7D4D0CDCAC6C3BFBC81
:10172700B8B4B0ACA8A39F9B96928D89847F7A7535
:10173700706B66615C57514C47413C37312C262111
:101747001B16100B050000050B10161C21272C3249
:10175700373D42484D53585D62686D72777C81858D
:101767008A8F94989DA1A5AAAEB2B6BABEC1C5C8C4
:10177700CCCFD2D5D8DBDEE1E3E6E8EBEDEFF1F253
:10178700F4F6F7F8F9FBFBFCFDFEFEFEFEFE000C8F
:101797001926333F4C5864707B86919CA6AFB8C11D
:1017A700C9D1D8DEE4EAEFF3F6F9FCFDFEFEFEFD53
:1017B700FCFAF7F4F0EBE6E0DAD4CCC5BCB4ABA1A5
:0E17C700978D83786D61554A3D3125180C00D1
:101DCC00D2F4C2F5C2F675840F85F0C81224B6742D
:101DDC0003121E1B1224AA7403121E1B12248D1232
:101DEC00248D7403121E1B12248D7402121E1B12DE
:101DFC00248D7428121E877406121E87740E121EF0
:101E0C00877401121E871224AA7480121E8722C0A6
:101E1C0000A2E092F3A2E192F2A2E292F1A2E3928A
:101E2C00F0D2F475840F85F0C8C2F47830D8FE85F2
:101E3C00F0C87830D8FED00022C00075840FA2E420
:101E4C0092F3A2E592F2A2E692F1A2E792F0D2F41A
:101E5C0085F0C8C2F47830D8FE85F0C87830D8FE4A
:101E6C00D00022EF75840FD2F5C2F685F0C8121E91
:101E7C004512248D121E1B12248D2275840FC2F55F
:101E8C00C2F685F0C8121E4512248D121E1B122498
:101E9C008D22EF14A2E492E6C2E4D2E7121E87224E
:101EAC00740F121E8722740D121E87227F01121EC0
:101EBC009E78107F20121E6FD8F9227F11121E9E61
:101ECC0078107F20121E6FD8F9227F01121E9E7887
:101EDC00207F20121E6FD8F922C0077F018004C01A
:101EEC00077F11121E9ED007C082C083C007EF75FA
:101EFC00F010901F161224CE7810E493FF121E6F70
:091F0C00A3D8F7D007D083D082DE
:101F150022202020202020202020202020202020BA
:101F25002057414954494E4720464F522052494E69
:101F3500472054454C434F20414E53574552454445
:101F450020205741495420464F5220444953434F7E
:101F55002020205445535420204641494C454420D7
:101F650020202054455354202050415353454420AC
:101F7500202020454550524F4D2054455354202094
:101F850020204155582052454C4159205445535421
:101F95002020205055534820544F2054414C4B206D
:101FA5002054455354203320434841522F53554222
:101FB50020544553542046495845442053545249CA
:101FC5004E54455354205641524942205354524988
:101FD5004E464143544F52592044454641554C5471
:101FE5002050524F4752414D4D494E47204D4F4489
:101FF5004553494D504C455820524550454154454F
:10200500522020205245434F5244494E472020201C
:0120150020AA
:102A320032C28D32758400C2CF32C0E0C083C08200
:102A4200C0D0C000C0F0C2CFB21A201A2312142480
:102A5200151BE51B7009751B0A7584017588AF1576
:102A62001CE51C7009751C607584027588AF8011A5
:102A72001215AC1536E5367008753604758400D229
:102A82008B758400D2ECD0F0D000D0D0D082D0832D
:102A9200D0E032C2CF32C0E0C0D0C007C000C08395
:102AA200C08212439E75888FD082D083D000D00717
:102AB200D0D0D0E032C0E0C0D0C000C083C082C05D
:102AC2008420121375840F30DF27E5E8540FF54098
:102AD200D2127541C8801A1541E5417006E540D20F
:102AE200E7F54075840F20DF08C212D211D22AD234
:102AF2002D20141475840F30F828E5E854F0C4F53D
:102B020042D2147543C8801A1543E5437006E54264
:102B1200D2E7F54275840F20F808C214D213D229E5
:102B2200D21C1243E3151DE51D702A751D0A1244BD
:102B32000A151EE51E701E751E0A12445D151FE55C
:102B42001F7012751F0612445E1526E52670067563
:102B5200260A124467D084C28DD082D083D000D09E
:102B6200D0D0E0323220100DD21085BF3585BE3470
:0A2B720075BB01800BC21085BF3354
:102B7C0085BE3275BB00C2ED32C0E0C0D0E544B4B6
:102B8C00000A054485BE3F75BB07803DB4010A05AC
:102B9C004485BE3C75BB048030B4020A054485BE36
:102BAC003F75BB068023B4030A054485BE3D75BB47
:102BBC00048016B4040A054485BE3F75BB05800924
:102BCC0075440085BE3E75BB04C2EDD0D0D0E0325A
:103DC50044313233343536373839302A234142438A
:103DD500202020205354414E4442592020202020A9
:103DE500524144494F204F524947494E415445207D
:103DF50054454C434F204F524947494E4154452065
:103E050020202046554E4354494F4E203120202036
:103E150020202046554E4354494F4E203220202025
:103E250020202046554E4354494F4E203320202014
:103E350020202046554E4354494F4E203420202003
:103E450020202046554E4354494F4E2035202020F2
:103E550020202046554E4354494F4E2036202020E1
:103E650020202046554E4354494F4E2037202020D0
:103E750020202046554E4354494F4E2038202020BF
:103E850020202046554E4354494F4E2039202020AE
:103E9500202052454345495645204D4F4445202055
:103EA500205452414E534D4954204D4F44452020F6
:103EB500202045204C4541442044454C4159202073
:103EC500205741495420464F52204D204C454144EE
:104470001267541249FC75840F1200A41267481287
:10448000608E1260C71263C012580320A503120E7B
:10449000DA9000A5E4F020A432302915C229E542C3
:1044A000540FFFEF903DC593FF90008CEFF0124E3C
:1044B000E1302AE2C22AE540540FFFEF903DC59358
:1044C000FF90008BEFF0124FC480CB9000A5E0FF6F
:1044D000EF1241A144F90044FE01450302450803DF
:1044E000450D04451205451806451E074524084597
:1044F0002A0945300A00004496125B8A80981245CA
:10450000FA809312560D808E1263ED8089122BDC97
:104510008084122F1D024496124F53024496125E5D
:10452000F2024496125A6702449612659A02449621
:0A453000124B170244960244962233
:105B8A0012658012673C1267481266521263351218
:105B9A0063C0125C5D12680A9000ACE4F09000B138
:105BAA00E4F09000A6E4F09000EEE4F09000EDE45A
:105BBA00F07BFF7A3D79D51262A9121EC775383279
:075BCA009000A5E004F022A9
:1045FA00E53860030246B812481B125381302B0B70
:10460A00126490C22B9000A5E4F022301F0B1261B5
:10461A0000C21F9000A5E4F02212661C50409000D0
:10462A00E1E0FF9000A7EFF09000EBE0FFEFB402AB
:10463A00031267369000ECE0FFEFB4020312674200
:10464A009000B1E4F07BFF7A3D79F51262A97BFF15
:10465A007A3E79B51262DA9000A57402F0221266E7
:10466A002EEF604A9000EAE0FFEF60421266629025
:10467A0000E2E0FF9000A8EFF09000EBE0FFEFB45B
:10468A0002031267369000ECE0FFEFB402031267F0
:10469A00429000B1E4F07BFF7A3D79E51262A97B92
:0F46AA00FF7A3E79C51262DA9000A57406F022FD
:10560D00121B759000A7E0FFEF702D1266629000DF
:10561D00EBE0FFEFB402031267369000ECE0FFEF12
:10562D00B4020312674275370A7BFF7A3E799512F1
:10563D0062DA9000A57403F012481B302B0B126434
:10564D0090C22B9000A5E4F022301F0A126100C217
:07565D001F9000A5E4F022FC
:1063ED00121B75E53770231267F21267BF126580B5
:1063FD009000D8E0FF9000A3EFF09000EDE4F09056
:0B640D0000EEE4F09000A57405F02202
:102BDC0020A6031252511267BC121B751217D51284
:102BEC005112125381123ED512481B9000EEE0FF99
:102BFC00EF603F1265801266529000EBE0FFEF64CD
:102C0C000160099000EBE0FFEFB4020312673C9007
:102C1C0000ECE0FFEF640160099000ECE0FFEFB422
:102C2C0002031267489000EF740AF09000A5740933
:102C3C00F0229000DBE0FFEF705C9000A6E0FFEF6D
:102C4C00602B900098E0FFEF70239000A6E4F090CA
:102C5C000099E4F09000DEE0FF9000D9E0FEEE2F4A
:102C6C00FF9000A1EFF09000A5740AF0229000985C
:102C7C00E0FFEF702190009CE0FFEF70199000DEF8
:102C8C00E0FF9000D9E0FEEE2FFF9000A1EFF09056
:102C9C0000A5740AF0229000DBE0FFEFB401219054
:102CAC000098E0FFEF70199000DEE0FF9000D9E093
:102CBC00FEEE2FFF9000A1EFF09000A5740AF02219
:102CCC009000DBE0FFEFB4022190009CE0FFEF707E
:102CDC00199000DEE0FF9000D9E0FEEE2FFF90008F
:102CEC00A1EFF09000A5740AF0229000DBE0FFEF5A
:102CFC00D3940240219000B1E0FFEF70199000DEF8
:102D0C00E0FF9000D9E0FEEE2FFF9000A1EFF090D5
:102D1C0000A5740AF022302B2012658012673C1239
:102D2C006748126652126490C22B1267DD1267E379
:102D3C001267BF9000A5E4F022301F1D12658012AF
:102D4C00673C1267481267DD1267E31267BF1261B6
:102D5C0000C21F9000A5E4F02212661C40189000DF
:102D6C00DEE0FF9000D9E0FEEE2FFF9000A1EFF027
:072D7C009000A57408F0228D
:102F1D0020A6031252511266911264DE121B751215
:102F2D0017D51267E31267DD125112125381123E4B
:102F3D00D512481B9000EEE0FFEF603F1265801246
:102F4D0066529000EBE0FFEF640160099000EBE04A
:102F5D00FFEFB4020312673C9000ECE0FFEF640159
:102F6D0060099000ECE0FFEFB40203126748900097
:102F7D00EF740AF09000A57409F0229000DBE0FFD9
:102F8D00EF701A900098E0FFEF700E90009CE0FF3C
:102F9D00EF600A12662EEF7004125C18229000DBAF
:102FAD00E0FFEFB4010C900098E0FFEF6004125CBD
:102FBD0018229000DBE0FFEFB4021290009CE0FFBE
:102FCD00EF600A12662EEF7004125C18229000DB7F
:102FDD00E0FFEFB4030C9000B1E0FFEF6004125C72
:102FED0018229000DBE0FFEFB4040C9000B1E0FF7D
:102FFD00EF6004125C1822302B2012658012673CA2
:10300D001267481266521267F51264901267DD124C
:10301D0067F5C22B9000A5E4F022301F1D126580CC
:10302D0012673C1267481267DD1267BF1267F5120F
:10303D006100C21F9000A5E4F02212661C404012F0
:10304D0066521265809000EBE0FFEF64016009901D
:10305D0000EBE0FFEFB4020312673C9000ECE0FFE1
:10306D00EF640160099000ECE0FFEFB4020312671A
:10307D00481267DD1267E31267BF9000A5E4F022E6
:104F530012538112662EEF600A9000E2E0FF900088
:104F6300A8EFF09000A8E0FFEF70299000E2E0FFC7
:104F7300EF60211266529000EBE0FFEFB4020312E0
:104F8300673C9000ECE0FFEFB40203126748900027
:104F9300A5E4F02212661C500975370A9000A57427
:104FA30007F012481B302B0B126490C22B9000A504
:104FB300E4F022301F0A126100C21F9000A5E4F042
:014FC30022CB
:105EF20012661C400375370AE537701275370A7B44
:105F0200FF7A3E79951262DA9000A57403F0124886
:105F12001B302B0B126490C22B9000A5E4F02230B0
:0D5F22001F0A126100C21F9000A5E4F022CA
:105A67009000A1E0FFEF704012665212658090002F
:105A7700EBE0FFEF640160099000EBE0FFEFB40299
:105A87000312673C9000ECE0FFEF640160099000AF
:105A9700ECE0FFEFB402031267481267DD1267E319
:095AA7001267BF9000A5E4F02293
:10659A009000EFE0FFEF700E1267DD1267E31267FB
:0765AA00BF9000A5E4F02200
:104B17009000A1E0FFEF7004126272221267BC12CC
:104B27001B751217D5123ED512481B302B0B12647A
:104B370090C22B9000A5E4F022301F0B126100C237
:104B47001F9000A5E4F0229000EEE0FFEF603E1218
:104B570065801266529000EBE0FFEF6401600990F8
:104B670000EBE0FFEFB4020312673C9000ECE0FFBC
:104B7700EF640160099000ECE0FFEFB402031267F5
:0E4B8700489000EF740AF09000A57409F02227
:105C18001267F512680D125BD11267BF9000E8E0B9
:105C2800FFEF60069000AE7401F01265669000EB1D
:105C3800E0FFEFB401031267369000ECE0FFEFB429
:105C480001031267427BFF7A3E79A51262DA90005F
:055C5800A57404F02218
:106272007BFF7A3E79951262DA1267BF1267F212D9
:1062820065809000EBE0FFEFB4010312673C9000E1
:10629200ECE0FFEFB401031267489000A57405F02B
:0162A20022D9
:106652009000E0E0FFEF600412674E2212675422BE
:106662009000E0E0FFEF60041267542212674E22AE
:10661C009000DFE0FFEF600612677EB32222126764
:02662C007E22CC
:103FD600900091E0FF703B9000CAE060159000CB26
:103FE600E0FEE53ED39E40249000CCE09000930294
:103FF600408E9000CBE0FEE53EC39E500F9000CC75
:10400600E0900093F09000917403F022E490009405
:10401600F022EF640170249000CBE024FBFFE53E24
:10402600D39F406C900093E060030240D1900094CF
:1040360004F09000CDE0900092804D900091E0FF5A
:10404600B402179000CBE024FBFEE53ED39E40026F
:10405600805F900092E070738066EF640370339027
:1040660000CBE02405FFE433FEC3E53E9FEE64800B
:10407600F8748098501A900093E0704F9000940462
:10408600F09000CDE0900092F0900091E004F022D4
:104096008034900091E06404702C9000CBE02405FD
:1040A600FFE433FEC3E53E9FEE6480F874809850CB
:1040B600099000CDE0900092F022900092E0700B03
:0C40C600900094F08001E4900091F02242
:10532000900091E0700E12675A50559000CCE090BA
:105330000093801E900091E0B4012212675A501A27
:10534000900093E0701790009404F09000CDE090EE
:105350000092F0900091E004F022E4801F90009110
:10536000E0B4021C12675A50099000CDE090009200
:10537000F022900092E07008900094F0900091F07C
:01538000220A
:0D6691009000C9E06003025320123FD622A2
:103ED500900095E0FF703B9000CEE060159000CF1C
:103EE500E0FEE53DD39E40249000D0E0900097028F
:103EF5003F959000CFE0FEE53DC39E500F9000D06A
:103F0500E0900097F09000957403F022E4900098FB
:103F1500F022EF640170259000CFE024FBFFE53D22
:103F2500D39F4074900097E0701290009804F09031
:103F350000A6F09000D1E09000968054900095E0A6
:103F4500B402179000CFE024FBFFE53DD39F40026C
:103F55008064900096E07002806B900095E0FF64AD
:103F65000370379000CFE02405FDE433FCE53DC345
:103F75009DEC6480F8748098501E900097E0701A4C
:103F850090009804F09000A6F09000D1E090009683
:103F9500F0900095E004F0228031EF6404702C90DD
:103FA50000CFE02405FFE433FEC3E53D9FEE6480CA
:103FB500F874809850099000D1E0900096F0229016
:103FC5000096E07006900098F08001E4900095F06E
:013FD50022C9
:10511200900099E07019126766500E9000D4E090EA
:10512200009BF0900099E004F0E490009CF0229043
:105132000099E0B40122126766501A90009BE07059
:105142001790009C04F09000D5E090009AF0900037
:1051520099E004F022E4801F900099E0B4021C124E
:10516200676650099000D5E090009AF02290009A6C
:0C517200E0700890009CF0900099F02282
:1053810090009DE0700E12676050559000D2E09041
:10539100009F801E90009DE0B40122126760501AA8
:1053A10090009FE070179000A004F09000D3E0906F
:1053B100009EF090009DE004F022E4801F90009D8B
:1053C100E0B4021C12676050099000D3E090009E87
:1053D100F02290009EE070089000A0F090009DF0F7
:0153E10022A9
:10662E009000D7E060069000A0E0FF22900094E07A
:02663E00FF2239
:1064DE009000D8E0FF601D90009CE070069000A038
:1064EE00E060069000A3EFF0229000A3E07005900C
:0564FE00009004F022F3
:104E6E0054564F582020434F53202053454E534500
:104E7E00004F4E20202020202020202020202020E7
:104E8E0020004F46462020202020202020202020B9
:104E9E00202000191823A01296203D129623A0124E
:104EAE009627631488203D148823A0148827631640
:104EBE00B8203D16B823A016B827631918203D193F
:104ECE0018276312962B8C14882B8C16B82B8C19E2
:034EDE00182B8C02
:1049FC0012679812679512675AE433F54F12679B4A
:104A0C00E433F54F12679EE433F54F1267A1E4339C
:104A1C00F54F1267A4E433F54F1267A7E433F54F53
:104A2C001267AAE433F54F1267ADE433F54F126702
:104A3C00B0E433F54F12676CE433F54F1267B3E40F
:104A4C0033F54F126778E433F54F1267B61267B936
:104A5C001267C21267C51267C81267CB1267CE12F3
:104A6C0067D11267D41267D71267E61267E912672B
:104A7C00EC1267EF1267F81267FB1267FE126801FF
:064A8C0012680402680735
:0667360075840FD2FC2265
:06673C0075840FC2FC226F
:0667420075840FD2B7229E
:0667480075840FC2B722A8
:06674E0075840FD2FE224B
:0667540075840FC2FE2255
:1065660075840FD2FD9000EBE0B4010312673690FC
:0A65760000ECE0B4010312674222BA
:1065800075840FC2FD9000EBE0B4010312673C90EC
:0A65900000ECE0B40103126748229A
:03679500C293228A
:03679800D2932277
:06675A0075840FA2FA2273
:03679B00A2A02297
:03679E00A2A12293
:0367A100A2A2228F
:0367A400A2A3228B
:0367A700A2A42287
:0367AA00A2A52283
:0367AD00A2A6227F
:0367B000A2A7227B
:0667600075840FA2F9226E
:0667660075840FA2DD2284
:06676C0075840FA2DE227D
:0367B300A292228D
:0667720075840FA2DA227B
:0667780075840FA2DB2274
:06677E0075840FA2DC226D
:0667840075840FA2D8226B
:06678A0075840FA2D92264
:0367B600D20822E4
:0367B900C20822F1
:0367BC00D20922DD
:0367BF00C20922EA
:0367C200D20A22D6
:0367C500C20A22E3
:0367C800D20222D8
:0367CB00C20222E5
:0367CE00D20B22C9
:0367D100C20B22D6
:0367D400D20C22C2
:0367D700C20C22CF
:0367DA00D20D22BB
:0367DD00C20D22C8
:0367E000D21822AA
:0367E300C21822B7
:0367E600D20E22AE
:0367E900C20E22BB
:0367EC00D20F22A7
:0367EF00C20F22B4
:0367F200D20022B0
:0367F500C20022BD
:0367F800D20122A9
:0367FB00C20122B6
:0367FE00D20322A1
:03680100C20322AD
:03680400D2042299
:03680700C20422A6
:105BD100E4FDFCED25E0FFEC33FE74002FF582744B
:105BE100023EF583E4F0A3F00DBD00010CBC0EE311
:105BF100BDE0E07558027559007402F55AF55B90E5
:105C010000D9E075F0BEA4AEF02400F55DEE3402DB
:065C1100F55CC200D205A3
:015C1700226A
:03680A00C20522A2
:105C5D00E4FDFCED25E0FFEC33FE74002FF58274BE
:105C6D00023EF583E4F0A3F00DBD00010CBC0EE384
:105C7D00BDE0E07558027559007402F55AF55B9058
:105C8D0000D9E075F0BEA4AEF02400F55DEE34024F
:045C9D00F55CD206DA
:015CA10022E0
:03680D00C206229E
:0B66CE0075081575095ED215D2032275
:0B66D90075081575095ED215D20B2262
:07672800C215C203C20B22DF
:0B66E4009000BD1231F8D216D2042243
:0B66EF009000BE1231F8D216D20C222F
:0C31F800E0F529E4F512F513F514F515C7
:10320400EF1241A132FF2332EE2A323C30324E31EA
:1032140032603232723332843432963532A83632E6
:10322400BA3732CC3832DD393310413321423332AC
:10323400433343440000335B904EA1E493F50D7493
:103244000193F50E904EA3023352904EA5E493F5EC
:103254000D740193F50E904EA7023352904EA9E4DB
:1032640093F50D740193F50E904EAB023352904ECC
:10327400ADE493F50D740193F50E904EAF02335205
:10328400904EB1E493F50D740193F50E904EB30294
:103294003352904EB5E493F50D740193F50E904EB0
:1032A400B7023352904EB9E493F50D740193F50EC1
:1032B400904EBB023352904EBDE493F50D740193CE
:1032C400F50E904EBF023352904EC1E493F50D7447
:1032D4000193F50E904EC38075904EC5E493F50DA1
:1032E400740193F50E904EC78064904EC9E493F533
:1032F4000D740193F50E904ECB8053904ECDE49314
:10330400F50D740193F50E904ECF8042904ED1E4AA
:1033140093F50D740193F50E904ED38031904ED5F4
:10332400E493F50D740193F50E904ED78020904EE2
:10333400D9E493F50D740193F50E904EDB800F9054
:103344004EDDE493F50D740193F50E904EDFE49396
:08335400F50F740193F510223E
:07672F00C216C20CC20422D5
:05679000C215C2032246
:0B66FA007508027509ABD215D20B2207
:0B67050075081A7509ABD215D20B22E3
:105251001251121253817BFF7A4E796E1262A9901C
:10526100009CE07BFF60067A4E797F80047A4E795C
:10527100901262DA7F17121E9EAF3E122513900024
:105281006CE0FF121E6F90006DE0FF121E6F900028
:105291006EE0FF121E6F7F1C121E9EAF3D12251382
:1052A10090006CE0FF121E6F90006DE0FF121E6F08
:0852B10090006EE0FF021E6F89
:10024D0020202020202020202020202020202020A1
:10025D002020202020202020202020202020202091
:10026D002054454C434F2050524F4752414D202072
:10027D0020524144494F2050524F4752414D20206A
:10028D002050484F4E452050524F4752414D20204F
:10029D0020434F4D50552050524F4752414D202035
:1002AD00202041434345535320434F4445202020B4
:1002BD0044544D462054454C434F204C4556454CD7
:1002CD0044544D4620524144494F204C4556454CCF
:1002DD004245455020524144494F204C4556454CCE
:1002ED00424545502054454C434F204C4556454CB6
:1002FD0054454C434F20524144494F204C45564C98
:10030D00524144494F2054454C434F204C45564C87
:10031D00524144494F204C494D4954204C45564C6F
:10032D002045494120544F4E45204C4556454C20C3
:10033D004C4F57204755415244204C4556454C2073
:10034D0048494748204755415244204C4556454C55
:10035D00564F494345205241444930204C45564C57
:10036D00564F4943452054454C434F204C45564C20
:10037D0020434F53204F5220535155454C43482055
:10038D002020434F5320504F4C4152495459202067
:10039D00434F53205452494747455220564F4C54D2
:1003AD00434F5320414351554953542054494D45D2
:1003BD00434F532052454C454153452054494D45DB
:1003CD002053454E534520504F4C415249545920CE
:1003DD0053454E205452494747455220564F4C5491
:1003ED0053454E20414351554953542054494D4591
:1003FD0053454E2052454C454153452054494D459A
:10040D005220564F582041435155495354494F4E50
:10041D0020525820564F582052454C4541534520A7
:10042D005420564F582041435155495354494F4E2E
:10043D0020545820564F582052454C454153452085
:10044D00204F5045524154494E47204D4F44452071
:10045D0020564F58204F5220434152524945522069
:10046D002020564F58204143544956495459202075
:10047D00202054454C434F2044454C4159202020C9
:10048D002020524144494F2044454C4159202020C1
:10049D0053454E53452C20564F582C20544F4E4506
:1004AD0020204143434553532044454C415920207E
:1004BD00205455524E204F4E2044454C415920203A
:1004CD00205455524E204F46462044454C4159200C
:1004DD004449474954414C20494E20504F4C4152BC
:1004ED00434E544C2052454C415920504F4C415293
:1004FD002020452D44454C41592050425820202064
:10050D002020452D44454C41592052454320202063
:10051D00202052494E474F5554204D4F44452020E1
:10052D00414E535745522052494E47204E4D42524F
:10053D0020202052494E4720535041434520202032
:10054D00202052494E4720414E53574552202020DE
:10055D0052494E47205452414E534954494F4E53E0
:10056D0045494120544F4E4520454E41424C452072
:10057D0046554E4354494F4E20382053454C454324
:10058D00524144494F2053454C454320454E424C22
:10059D00204155582052454C4159204D4F4445203E
:1005AD002043542052454C4159204D4F4445202065
:1005BD00202020202020202020202020202020202E
:1005CD00202020202020202020202020313D454E9D
:1005DD002020202020202020202020524154494F2F
:1005ED002020202020202020202020303D434F534C
:1005FD002020202020202020202020313D504F532E
:10060D0020202020202020202020202031204D536C
:10061D0020202020202020202020203130204D534C
:10062D0020202020202020202020313030204D532C
:10063D002020202020202020202020202053454332
:10064D00202020202020202020202020204D494E19
:10065D002020202020202020202020204D4F4445E8
:10066D002020202020202020202020313D564F58B2
:10067D00202020202020202020202052494E47538A
:10068D0020202020202020202020204359434C458D
:10069D0020202020202020202020313D544F4E4569
:1006AD002020202020202020504F4C4152495459C9
:1006BD008201001102381500018201011103381564
:1006CD000001820102110438150001820103110598
:1006DD003815000178060411060119000082030A7D
:1006ED001107391500FF82030B1108391500FF8220
:1006FD00030C1109391500FF82030D110A3915007C
:10070D00FF82030E110B391500FF82030F110C39F7
:10071D001500FF820310110D391500FF8203111111
:10072D000E391500FF820312110F391500FF8203D8
:10073D00131110391500FF8203141111391500FF23
:10074D008203151112391500FF82011611133A1586
:10075D00000182011711143B1500018203181115B8
:10076D00391500FF82021911163C15006382021A19
:10077D0011173D15006382011B11183B15000182F5
:10078D00031C1119391500FF82021D111A3C1500A9
:10079D006382021E111B3D15006382021F111C3C5A
:1007AD00150063820220111D3E1500638202211186
:1007BD001E3C150063820222111F3E15006382014B
:1007CD00231120411500028201241121421500013F
:1007DD0082022511224015006382022611233D1548
:1007ED00002882022711243D150028820128112599
:1007FD004115000482022911263E150A6382022A40
:10080D0011273C15006382022B11283D15006382D0
:10081D00012C11294615000182012D112A461500C2
:10082D000182022E112B3D1501FF82022F112C3E4C
:10083D00150063820130112D3C150001820131112B
:10084D002E43150009820232112F3C1500638201DF
:10085D00331130411500018203341131441501FF6C
:10086D0082013511323815000182013611334515DB
:10087D00000182013711343815000182013811351C
:10088D004115000382013911364115000320202046
:10089D002020202020202020202020202082010127
:1008AD0011020C15000120202020202020202020C6
:1008BD0020202020202082010111020C1500012092
:1008CD0020202020202020202020202020202064D7
:1008DD0001001102091500012020202020202020D8
:1008ED0020202020202020200101010101010101F3
:1008FD0001000000000000000000000000000000EA
:10090D0000000000000000000000000000000000DA
:10091D0000000000000000000000000000000000CA
:10092D0000000000000000000000000000000000BA
:10093D0000000000000000000000000000000000AA
:10094D0000002020202020202020202020202020DA
:10095D002020010101010101010101000000000041
:10096D00000000000000000000000000000000007A
:10097D00000000000000000000000000000000006A
:10098D00000000000000000000000000000000005A
:10099D00000000000000000000000000000000004A
:1009AD0000000000000000000000000020202020BA
:1009BD0020202020202020202020202001010101A6
:1009CD000101010101000000000000000000000015
:1009DD00000000000000000000000000000000000A
:1009ED0000000000000000000000000000000000FA
:1009FD0000000000000000000000000000000000EA
:100A0D0000000000000000000000000000000000D9
:100A1D000000000000002020202020202020202089
:100A2D0020202020202082010011021E150001012E
:100A3D00010101313233343536FF323232FFFFFFDF
:100A4D00550CFF3232000180000A0080000A000AB6
:100A5D00000A0001002828001E140000012863016F
:100A6D000163000A01010102000000000000000006
:100A7D0044313233343536373839302A2341424305
:100A8D0044AAA3C1C2C3C4D7ABA8A92A23414243D8
:100A9D0036333036373036393437313937343437F9
:100AAD0037303739373832353835343838353931DC
:100ABD0035393438393734313030313033313037EE
:100ACD0031313031313431313831323331323731F6
:100ADD0033313133363134313134363135313135DD
:100AED0036313539313632313635313637313731B8
:100AFD0031373331373731373931383331383631A2
:100B0D003839313932313936313939323033323091
:100B1D003632313032313832323532323932333396
:100B2D003234313235303235343030363030373092
:100B3D003135303137303231303233303235303289
:100B4D00363033313033323033363034333034376E
:100B5D003035303035313035333035343036353061
:100B6D00373130373230373330373431313431314A
:100B7D003531313631323231323531333131333243
:100B8D00313334313431313433313435313532312F
:100B9D00353531353631363231363531373231370B
:100BAD003432303532313232313432323332323511
:100BBD0032323632343332343432343532343632F2
:100BCD0035313235323235353236313236333236E1
:100BDD0035323636323731323734333036333131D0
:100BED0033313533323533333133333233343333C9
:100BFD0034363335313335363336343336353337A2
:100C0D0031343131343132343133343233343331B0
:100C1D003433323434353434363435323435343487
:100C2D00353534363234363434363534363635306F
:100C3D00333530363531363532333532363533326C
:100C4D003534363536353630363631323632343651
:100C5D003237363331363332363534363632363640
:100C6D00343730333731323732333733313733323C
:100C7D0037333437343337353441424344454647AF
:100C8D0048494A4B4C4D4E4F50515253545556575F
:100C9D0058595A6162636465666768696A6B6C6D01
:100CAD006E6F707172737475767778797A303132C0
:100CBD0033343536373839607E21402324255E267E
:100CCD002A28295F2D2B3D7B7D5B5D7C3A3B3C3E8D
:100CDD002C2E3F2F202020202020202020202020BF
:100CED0020474C4F42414C202020202020204354AF
:100CFD0043535320434F444520202020202020449F
:100D0D00435320434F44452020202020204C545253
:100D1D0020524550454154455220202020535045E6
:100D2D004544204449414C494E47202020535045CD
:100D3D0045442043414C4C494E47202020205054DF
:100D4D0043204E554D424552202020202020564F05
:100D5D00494345204D455353414745532020564F58
:100D6D0049434520504C41594241434B2020204995
:100D7D004E56414C49442054595045202020204F77
:100D8D005554204F462052414E4745202020494C76
:100D9D004C4547414C2056414C554520204D55530F
:100DAD00542046494C4C204649454C44202020496E
:100DBD004C4C4547414C20434F4445202020444155
:100DCD00544120414343455054454420204C494E05
:100DDD0045204E554D4245523A2020202055534531
:100DED00522050524F4752414D4D494E4755534554
:100DFD00522049443A2020202020202020564F49BF
:100E0D004345205245434F5244494E472020494CBB
:100E1D004C4547414C20454E545259202020494CB9
:100E2D004C4547414C2047414E4720202020202053
:100E3D00434F4D504C455445442020202020474CD5
:100E4D004F42414C20454550524F4D2020202043CC
:100E5D005443535320454550524F4D2020202020C0
:100E6D0044435320454550524F4D202020202020F3
:100E7D004C545220454550524F4D2020202044497E
:100E8D00414C494E4720454550524F4D202043413E
:100E9D004C4C494E4720454550524F4D2020202067
:100EAD0050544320454550524F4D2020202052454F
:100EBD0050454154455220454550524F4D202049F3
:0D0ECD004E495449414C495A494E47202096
:106100009000A47464F0E4900000F030200B301F85
:1061100024125DB112268680F530210B301F161235
:106120005DF312268680F530220B301F0812287F7F
:0661300012268680F52214
:102686009000A4E07012900000E0D394004009C2CC
:1026960020C221C222C21F22900000E01241A127BF
:1026A6009F0027A20127A50227A80327AB0427AD71
:1026B6000527AF0627B10727B40827B70A27BA0B9D
:1026C60027BD0F27C01027C31427C61527C91927EA
:1026D600CC1A27CF1B27D21E27D51F27D82327DBA7
:1026E6002427DE2827E12927E42D27E72E27EA2FAE
:1026F60027ED3027F03227F33327F53427F835272F
:10270600FB6427FE6528016628046728076E2809EA
:102716006F280B70284D71280D78280F7928117AAB
:10272600284D7B2813822815832817842819852885
:102736001C8C281F8D28218E28238F282696282931
:1027460097282B98282D992830A02833A12836A21F
:102756002838A3283BAA283DAB2840AC2842AD2800
:1027660045B42848B5284BB6284DB7284FBE285241
:10277600BF2855C02858C1284DC2285EF02861F1EF
:102786002864F22867FA286AFB286DFC2870FD2861
:1027960073FE2876FF00002879026640026547022C
:1027A6005CA2026442800480028000025A1D02304C
:1027B6008D02620B02335C0256BA0234AA02570E2D
:1027C6000235F8025E35025442023B300258A2023C
:1027D60037460258EE02389402593A0239E2026349
:1027E60064026055025AB01259D20255598000024D
:1027F60050A4025D6E025762025CE6026136025523
:10280600B380468032804B8040802280458007809E
:1028160026803F02598602453A801C80350257B30E
:10282600024B958008802B025E7402476B0250357E
:1028360080200246B98012024D0B8016023C7B02B4
:102846004C8F0251E8800B800C024D8402585302D3
:1028560048C7025F2F02566402646902517E02660F
:10286600720254FD02681902681A02681B024C12B1
:0928760002681CE4900000F0224D
:10664000E4900002F09000A47464F0900000E00474
:02665000F02236
:10654700121EB8121EC77BFF7A0D79EA1262A97F65
:0F65570011121E9EC226C223900000E004F02203
:105CA200302340900001E0FFC223BF2A079000008A
:105CB200E004F022EF6423702A7F23121E6F90000B
:105CC20002E004F0E0C394034013C220C221C222C6
:105CD200C21FE4900000F0126418021ED690000069
:035CE2007402F059
:015CE500229C
:106442007BFF7A0D79EA1262A9121EC77F11121E12
:106452009E12669EE490003CF07F2A121E6FC226B6
:07646200900000E004F022AD
:105A1D00302346900001E0F55EC223E55E642A6006
:105A2D0038AF5E1266825022AF5E121E6F90003C40
:105A3D00E02403F582E43400F583E55EF090003C4C
:105A4D00E004F0900000E004F0227BFF7A0E791A5A
:095A5D001262A990000074FAF035
:015A6600221D
:10308D002023030231F7900001E0FFC223BF2A077E
:10309D009000007403F022EF642360030231E81204
:1030AD001E6F900004E064397077A3E0643970718D
:1030BD00A3E06439706BD227900003E0FFB43108B0
:1030CD00E4900036F0023157EFB43208E490003747
:1030DD00F002316AEFB43302803E900003E0FFB49A
:1030ED003408E4900038F0023198EFB43508E490DC
:1030FD000039F00231AEEFB43608E490003AF00238
:10310D0031C4EFB437028010900003E0B438028070
:10311D0007900003E0B4390B7BFF7A0E792A023158
:10312D00EEC227900003E0FFB43016A3E0B43011D7
:10313D00A3E0B4300CA3E0B43007900000740AF0A3
:10314D0022EFB4310C1254A05007900000740FF010
:10315D0022900003E0B4320C1253E25007900000AD
:10316D007414F022900003E0B43311A3E0B4300CDA
:10317D0012652650079000007419F022900003E0AC
:10318D00B4340FA3E0B4300A1265C8900000741E69
:10319D00F022900003E0B4350FA3E0B4300A1265BD
:1031AD00DD9000007423F022900003E0B4360FA3ED
:1031BD00E0B4300A1265F29000007428F0229000FD
:1031CD0003E0B43716A3E0B43011A3E0B4300CA380
:1031DD00E0B43007900000742DF0227BFF7A0E7959
:0A31ED001A1262A990000074FAF0B3
:0131F70022B5
:10620B0090003B740BF090003C7407F0E490004955
:10621B00F090004A743AF0E490004BF07BFF7A0C5C
:10622B0079EA1262A91262D47F1E121E9E900000A0
:04623B007432F022A7
:10335C00124DF9D3900072E09434900071E0940017
:10336C00400A1262A390000074FAF022900071E0FF
:10337C00FEA3E0FF9006BD75F009124195EE75F0C5
:10338C0009A42583F583E493900040F09006BE7564
:10339C00F009EF124195EE75F009A42583F583E44D
:1033AC0093900041F0900071A3E09006BF75F00976
:1033BC00124195EE75F009A42583F583E4939000F2
:1033CC0042F09006C075F009EF124195EE75F009C8
:1033DC00A42583F583E493900043F0900071A3E05F
:1033EC009006C175F009124195EE75F009A425837C
:1033FC00F583E493FD900044F09006C275F009EF5C
:10340C00124195EE75F009A42583F583E4939000A1
:10341C0045F0900071A3E09006C375F00912419538
:10342C00EE75F009A42583F583E493900046F090A3
:10343C0006C475F009EF124195EE75F009A42583C9
:10344C00F583E493900047F0900071A3E09006C5DB
:10345C0075F009124195EE75F009A42583F583E406
:10346C0093900048F0ED6015900044E075F010A4C6
:10347C00244DF9740235F0FA7BFF1262A9900045D5
:10348C00E0FF601175F010A4244DF9740235F0FAC8
:0E349C007BFF1262DA900040E0900000F02208
:1056BA0090003B7410F090003C7407F0900049741D
:1056CA003AF0E490004AF0900036E090004BF07B0C
:1056DA00FF7A0C79FA1262A91262D47F0D121E9E09
:1056EA00900004E0FF121E6F900005E0FF121E6F8B
:1056FA00900006E0FF121E6F7F1E121E9E90000091
:04570A007432F022E3
:1034AA00124DF9D3900072E09400900071E09400FC
:1034BA00400A1262A390000074FAF022900071E0B0
:1034CA00FEA3E0FF9008AA75F009124195EE75F087
:1034DA0009A42583F583E493900040F09008AB7526
:1034EA00F009EF124195EE75F009A42583F583E4FE
:1034FA0093900041F0900071A3E09008AC75F00938
:10350A00124195EE75F009A42583F583E4939000A2
:10351A0042F09008AD75F009EF124195EE75F00989
:10352A00A42583F583E493900043F0900071A3E00F
:10353A009008AE75F009124195EE75F009A425833D
:10354A00F583E493FD900044F09008AF75F009EF1D
:10355A00124195EE75F009A42583F583E493900052
:10356A0045F0900071A3E09008B075F009124195FA
:10357A00EE75F009A42583F583E493900046F09054
:10358A0008B175F009EF124195EE75F009A425838B
:10359A00F583E493900047F0900071A3E09008B29D
:1035AA0075F009124195EE75F009A42583F583E4B7
:1035BA0093900048F0ED6015900044E075F010A477
:1035CA00249AF9740835F0FA7BFF1262A990004533
:1035DA00E0FF601175F010A4249AF9740835F0FA26
:0E35EA007BFF1262DA900040E0900000F022B9
:10570E0090003B7415F090003C7407F090004974C3
:10571E003AF0E490004AF0900037E090004BF07BB6
:10572E00FF7A0D790A1262A91262D47F0C121E9EA4
:10573E00900004E0FF121E6F900005E0FF121E6F36
:10574E00900006E0FF121E6F7F1E121E9E9000003C
:04575E007432F0228F
:1035F800124DF9D3900072E09400900071E09400AD
:10360800400A1262A390000074FAF022900071E060
:10361800FEA3E0FF9008C375F009124195EE75F01E
:1036280009A42583F583E493900040F09008C475BD
:10363800F009EF124195EE75F009A42583F583E4AE
:1036480093900041F0900071A3E09008C575F009CF
:10365800124195EE75F009A42583F583E493900053
:1036680042F09008C675F009EF124195EE75F00921
:10367800A42583F583E493900043F0900071A3E0C0
:103688009008C775F009124195EE75F009A42583D5
:10369800F583E493FD900044F09008C875F009EFB5
:1036A800124195EE75F009A42583F583E493900003
:1036B80045F0900071A3E09008C975F00912419592
:1036C800EE75F009A42583F583E493900046F09005
:1036D80008CA75F009EF124195EE75F009A4258323
:1036E800F583E493900047F0900071A3E09008CB35
:1036F80075F009124195EE75F009A42583F583E468
:1037080093900048F0ED6015900044E075F010A427
:1037180024B3F9740835F0FA7BFF1262A9900045CA
:10372800E0FF601175F010A424B3F9740835F0FABD
:0E3738007BFF1262DA900040E0900000F02269
:105E35007BFF7A0D791A1262A97BFF7A0D79FA1226
:105E450062DA7F0E121E9E900005E0FF121E6F9013
:105E55000006E0FF121E6F7F1A121E9E90003B7413
:0F5E65001AF090003C7404F09000007432F022A8
:105442003028079000007403F0221262D47F1E12EB
:105452001E9E1252B9900073E0FEA3E0FFD39400A7
:10546200EE9400402FEF94FBEE9400502790003B07
:10547200741BF090003C7407F0900049743AF0E419
:1054820090004AF0900035E01490004BF09000003C
:0E5492007432F0221262A390000074FAF0222D
:103B3000D3900072E09400900071E09400400A126B
:103B400062A390000074FAF022900071E0FEA3E0FE
:103B5000FF9008DC75F009124195EE75F009A42577
:103B600083F583E493900040F09008DD75F009EF51
:103B7000124195EE75F009A42583F583E493900036
:103B800041F0900071A3E09008DE75F009124195B4
:103B9000EE75F009A42583F583E493900042F0903C
:103BA00008DF75F009EF124195EE75F009A4258341
:103BB000F583E493900043F0900071A3E09008E057
:103BC00075F009124195EE75F009A42583F583E49B
:103BD00093FD900044F09008E175F009EF124195D3
:103BE000EE75F009A42583F583E493900045F090E9
:103BF0000071A3E09008E275F009124195EE75F0AE
:103C000009A42583F583E493900046F09008E375BA
:103C1000F009EF124195EE75F009A42583F583E4D0
:103C200093900047F0900071A3E09008E475F009CC
:103C3000124195EE75F009A42583F583E493900075
:103C400048F0ED6015900044E075F010A424CCF924
:103C5000740835F0FA7BFF1262A9900045E0FF601E
:103C60001175F010A424CCF9740835F0FA7BFF121A
:0B3C700062DA900040E0900000F022BB
:1058A20090003B741FF090003C7407F09000497424
:1058B2003AF0E490004AF0900038E090004BF07B20
:1058C200FF7A0D792A1262A91262D47F0F121E9EEC
:1058D200900005E0FF121E6F900006E0FF121E6F9F
:0C58E2007F1E121E9E9000007432F02207
:10374600124DF9D3900072E09400900071E094005D
:10375600400A1262A390000074FAF022900071E011
:10376600FEA3E0FF9008F575F009124195EE75F09D
:1037760009A42583F583E493900040F09008F6753C
:10378600F009EF124195EE75F009A42583F583E45F
:1037960093900041F0900071A3E09008F775F0094E
:1037A600124195EE75F009A42583F583E493900004
:1037B60042F09008F875F009EF124195EE75F009A0
:1037C600A42583F583E493900043F0900071A3E071
:1037D6009008F975F009124195EE75F009A4258354
:1037E600F583E493FD900044F09008FA75F009EF34
:1037F600124195EE75F009A42583F583E4939000B4
:1038060045F0900071A3E09008FB75F00912419510
:10381600EE75F009A42583F583E493900046F090B5
:1038260008FC75F009EF124195EE75F009A42583A1
:10383600F583E493900047F0900071A3E09008FDB3
:1038460075F009124195EE75F009A42583F583E418
:1038560093900048F0ED6015900044E075F010A4D8
:1038660024E5F9740835F0FA7BFF1262A990004549
:10387600E0FF601175F010A424E5F9740835F0FA3C
:0E3886007BFF1262DA900040E0900000F0221A
:1058EE0090003B7424F090003C7407F090004974D3
:1058FE003AF0E490004AF0900039E090004BF07BD3
:10590E00FF7A0D793A1262A91262D47F0F121E9E8F
:10591E00900005E0FF121E6F900006E0FF121E6F52
:0C592E007F1E121E9E9000007432F022BA
:10389400124DF9D3900072E09400900071E094000E
:1038A400400A1262A390000074FAF022900071E0C2
:1038B400FEA3E0FF90095F75F009124195EE75F0E3
:1038C40009A42583F583E493900040F09009607582
:1038D400F009EF124195EE75F009A42583F583E410
:1038E40093900041F0900071A3E090096175F00994
:1038F400124195EE75F009A42583F583E4939000B5
:1039040042F090096275F009EF124195EE75F009E5
:10391400A42583F583E493900043F0900071A3E021
:1039240090096375F009124195EE75F009A4258399
:10393400F583E493FD900044F090096475F009EF79
:10394400124195EE75F009A42583F583E493900064
:1039540045F0900071A3E090096575F00912419556
:10396400EE75F009A42583F583E493900046F09066
:10397400096675F009EF124195EE75F009A42583E7
:10398400F583E493900047F0900071A3E0900967F9
:1039940075F009124195EE75F009A42583F583E4C9
:1039A40093900048F0ED6015900044E075F010A489
:1039B400244FF9740935F0FA7BFF1262A99000458F
:1039C400E0FF601175F010A4244FF9740935F0FA82
:0E39D4007BFF1262DA900040E0900000F022CB
:10593A0090003B7429F090003C7407F09000497481
:10594A003AF0E490004AF090003AE090004BF07B85
:10595A00FF7A0D794A1262A91262D47F0D121E9E35
:10596A00900005E0FF121E6F900006E0FF121E6F06
:0C597A007F1E121E9E9000007432F0226E
:1039E200124DF9D3900072E09400900071E09400BF
:1039F200400A1262A390000074FAF022900071E073
:103A0200FEA3E0FF9009C975F009124195EE75F029
:103A120009A42583F583E493900040F09009CA75C8
:103A2200F009EF124195EE75F009A42583F583E4C0
:103A320093900041F0900071A3E09009CB75F009DA
:103A4200124195EE75F009A42583F583E493900065
:103A520042F09009CC75F009EF124195EE75F0092C
:103A6200A42583F583E493900043F0900071A3E0D2
:103A72009009CD75F009124195EE75F009A42583E0
:103A8200F583E493FD900044F09009CE75F009EFC0
:103A9200124195EE75F009A42583F583E493900015
:103AA20045F0900071A3E09009CF75F0091241959D
:103AB200EE75F009A42583F583E493900046F09017
:103AC20009D075F009EF124195EE75F009A425832E
:103AD200F583E493900047F0900071A3E09009D140
:103AE20075F009124195EE75F009A42583F583E47A
:103AF20093900048F0ED6015900044E075F010A43A
:103B020024B9F9740935F0FA7BFF1262A9900045D5
:103B1200E0FF601175F010A424B9F9740935F0FAC8
:0E3B22007BFF1262DA900040E0900000F0227B
:106364003022079000007401F02290003B742EF05C
:1063740090003C7407F07BFF7A0D795A1262A912DF
:0E63840062D47F1E121E9E9000007432F02222
:10605500302807900000742FF02290000AE0643881
:106065006005A3E0B4390A1262A390000074FAF047
:10607500227BFF7A0E790A1262A990000AE0540F7A
:09608500F5489000007430F0228F
:105AB00090000AE064386005A3E0B4390A1262A3DA
:105AC00090000074FAF0227BFF7A0D796A1262A9C5
:105AD00090000AE0540FF548D202D20A9000C8E0C4
:105AE000F527122D837BFF7A0E793A1262A9C20242
:095AF000C20A90000074FEF022CD
:1059D20090000AE0540FF548302002D200122D95B3
:1059E20030201B201304E53B70F9122D8CC2007B82
:1059F200FF7A0E793A1262A990000074FEF030210B
:105A020019201104E53B70F9122D8C7BFF7A0E7977
:0B5A12003A1262A990000074FEF0221E
:10555900302356900001E0FF900034F0C223121E60
:105569006F900034E0FF1266825021900034E0FF12
:1055790090003CE02403F582E43400F583EFF090D9
:10558900003CE004F0900000E004F022900034E0D8
:10559900B42A079000007403F0227BFF7A0E791A6F
:0A55A9001262A990000074FAF022CB
:1050A40030236A900001E0FF900034F0C223121E06
:1050B4006F900034E0FFB42A0B90003BE0900000B6
:1050C400F0D22822EFB4230B90003BE0900000F0D4
:1050D400C22822900034E0FF1266825021900034EE
:1050E400E0FF90003CE02403F582E43400F583EF14
:1050F400F090003CE004F0900000E004F0227BFF1C
:0E5104007A0E791A1262A990000074FAF02255
:105D6E0030233F900001E0FF900034F0121E6FC20E
:105D7E0023900034E0FFB42A0B90003BE09000002B
:105D8E00F0D22822EFB4230B90003BE0900000F0FD
:105D9E00C228227BFF7A0E791A1262A99000007433
:035DAE00FAF022E6
:0A576200900043E0FF700330283888
:10576C00121E9E1265031249A58F5E900041E052F5
:10577C005EE55E60047F3180027F30121E6F302840
:10578C0017C228E55E2430900023F090003374019A
:08579C00F090000074F0F0220F
:0F57A400900046E0FF121E9E900000E004F022ED
:105CE600302340900001E0FF900034F0C223121EE2
:105CF6006F900034E0FFB42A079000007403F0228E
:105D0600126682500F900034E090000DF090000073
:105D1600E004F0227BFF7A0E791A1262A990000045
:045D260074FAF022F9
:10613600302332900001E0FF900034F0C223BF2AE2
:10614600079000007403F022900034E0B423079017
:106156000000E004F0227BFF7A0E791A1262A99001
:06616600000074FAF022B3
:1055B300126503900075EEF0A3EFF01249A58F4F2B
:1055C30090003D7401F090000DE0B431089000416B
:1055D300E0424F800E90000DE0B4301E900041E099
:1055E300F4524F900075E0FEA3E0FFAD4F12496403
:1055F30012660790000074FEF0227BFF7A0E791A80
:0A5603001262A990000074FAF02270
:104D8400900043E0FF7003302856121E9E12650304
:104D9400900075EEF0A3EFF0E4F54F900041E0FFD2
:104DA400E54FC39F5027900075E475F00112417FD1
:104DB400AFF0FE1249A58F507423254FF582E434D9
:104DC40000F583E550F0121E6F054F80CE30281099
:104DD400C228E54F04900033F090000074F0F022F4
:104DE40090003C740AF0900046E0FF121E9E900072
:054DF40000E004F022C4
:104D0B00302375900001E0FF900034F0C223121E97
:104D1B006F900034E0FFB42A079000007403F02278
:104D2B00EFB42308900000E004F080391266825043
:104D3B0038900034E0FF90003CE0FE04F074032E4A
:104D4B00F582E43400F583EFF0900041E02409FF95
:104D5B00E433FE90003CE0D39FEE6480F8748098BF
:104D6B004016900000E004F0227BFF7A0E791A12B5
:094D7B0062A990000074FAF02214
:105F2F00302337900001E0FF900034F0C223121E9F
:105F3F006F900034E0FFB42A079000007403F02242
:105F4F00EFB42307900000E004F0227BFF7A0E7974
:0B5F5F001A1262A990000074FAF022F0
:10566400126503900075EEF0A3EFF090003C740A0D
:10567400F0E4F54F900041E0FFE54FC39F502790C1
:105684000075E475F00112417FAFF0FE90003CE03C
:10569400FD04F074032DF582E43400F583E0FD127B
:1056A4004964054F80CE7BFF7A0E793A1262A99045
:0656B400000074FEF0226C
:1050350030236B900001E0FF900034F0C223121E74
:105045006F900034E0FFB42A079000007403F0224B
:10505500126682501A900034E0FF90003CE0FE0496
:10506500F074032EF582E43400F583EFF080107BB5
:10507500FF7A0E791A1262A990000074FAF0229054
:105085000041E02409FFE433FE90003CE0D39FEEAD
:0F5095006480F87480984006900000E004F022D8
:10453A00900043E0FF70062028030245E5121E9E04
:10454A00126503900075EEF0A3EFF01249A512254B
:10455A0013900041E0B4011090006EE0FF121E6F4C
:10456A0090006EE0900023F0900041E0B4022090A9
:10457A00006DE0FF121E6F90006EE0FF121E6F903A
:10458A00006DE0900023F090006EE0900024F0901F
:10459A000041E06403703090006CE0FF121E6F90DF
:1045AA00006DE0FF121E6F90006EE0FF121E6F900A
:1045BA00006CE0900023F090006DE0900024F090F1
:1045CA00006EE0900025F0302811C228900041E0EA
:1045DA00900033F090000074F0F022900046E0FF63
:1045EA00121E9E90003C740AF0900000E004F02233
:105986001225695002803B1225418F4F900047E057
:10599600FFE54FC39F402B900048E0FFE54FD39FA4
:1059A6005020126503900075EEF0A3EFF0AD4F1294
:1059B60049647BFF7A0E793A1262A990000074FE60
:0C59C600F0221262A390000074FAF0229C
:1057B3001225695002803F1225418F4F900047E028
:1057C300FFE54FC39F400B900048E0FFE54FD39F99
:1057D3004004E54F7020126503900075EEF0A3EFCF
:1057E300F0AD4F1249647BFF7A0E793A1262A990A9
:1057F300000074FEF0221262A390000074FAF022FB
:104B9500900043E0FF700330285E121E9E126503ED
:104BA500900075EEF0A3EFF01249A58F4F124A92CF
:104BB500E4F54F746C254FF582E43400F583E0FF8E
:104BC5007423254FF582E43400F583EFF0746C25EA
:104BD5004FF582E43400F583E0FF121E6F054FE5C3
:104BE5004FC3940440CD30280FC22890003374037E
:104BF500F090000074F0F022900046E0FF121E9E37
:0D4C050090003C740AF0900000E004F022E2
:105E74007F0A1241C78F4FE54F60121265039000ED
:105E840075EEF0A3EFF0E54F14FD124964E54F7B86
:105E9400FF600E7A0E793A1262A990000074FEF047
:0F5EA400227A0D79BA1262A990000074FAF022E6
:10476B00900043E0FF7006202803024806121E9EAD
:10477B00126503900075EEF0A3EFF01249A5122518
:10478B0013900075E475F00112417FAFF0FE1249F2
:10479B00A51224F790006DE0FF900023F0A3F01218
:1047AB001E6F90006EE0FF121E6F900075E475F0A7
:1047BB000112417FAFF0FE1249A51224F790006C55
:1047CB00E0FF900025F090006DE0900026F0900047
:1047DB006EE0900027F0121E6F90006DE0FF121E2E
:1047EB006F90006EE0FF121E6F30280FC2289000F2
:1047FB00337405F090000074F0F022900046E0FF57
:10480B00121E9E90003C740AF0900000E004F0220F
:1046B90090000DE0540F75F00AA4FFA3E0540F2FEA
:1046C900F54F900010E0540F75F00AA4FF90000F09
:1046D900E0540F75F064A42FFF900011E0540F2FE0
:1046E900F550E54FC394014015E54FD39414500E8E
:1046F900E550C394014007E550D394FA400A126289
:10470900A390000074FAF022126503900075EEF090
:10471900A3EFF0900075E475F00112417FAFF0FE50
:10472900AD4F124964900010E0540F75F00AA4FFD0
:1047390090000FE0540F75F064A42FFF900011E072
:10474900540F2FF54F900075E0FEA3E0FFAD4F1217
:1047590049647BFF7A0E793A1262A990000074FECF
:02476900F0223C
:103C7B007F0D1241C7EF701A900010E0B43010A303
:103C8B00E0B4300BA3E0B43006A3E0643060030271
:103C9B003D65900014E0FF64306004EFB4350E9086
:103CAB000015E0540FD394054003023D65900014BA
:103CBB00E0FF64316004EFB43611900019E0B420DA
:103CCB0007900018E0B42003023D65900014E0FF5C
:103CDB0064326004EFB43710900018E0B420079002
:103CEB000017E0B420028072900014E0FF64336090
:103CFB0004EFB43809900015E0B42002805C90000A
:103D0B0014E0FF64346005EF64397058900015E0DF
:103D1B00540F75F00AA4FFA3E0540F2FF54F90003A
:103D2B0018E0540F75F00AA4FF900017E0540F75BC
:103D3B00F064A42FFF900019E0540F2FF550E54FBE
:103D4B00C394014015E54FD39414500EE550C39422
:103D5B00014007E550D394FA400A1262A390000089
:103D6B0074FAF022126503900075EEF0A3EFF09059
:103D7B00003C740AF0E4F54F900041E0FFE54FC3BF
:103D8B009F5027900075E475F00112417FAFF0FE54
:103D9B0090003CE0FD04F074032DF582E43400F553
:103DAB0083E0FD124964054F80CE7BFF7A0E793A92
:0A3DBB001262A990000074FEF022CD
:104C8F00900043E0FF700330285B121E9E126503F5
:104C9F00900075EEF0A3EFF0E4F54F900041E0FFC8
:104CAF00E54FC39F502C900075E475F00112417FC2
:104CBF00AFF0FE1249A58F507423254FF582E434CF
:104CCF0000F583E550F07E001249A5121E6F054FC7
:104CDF0080C9302810C228E54F04900033F09000AF
:104CEF000074F0F022900046E0FF121E9E90003CF0
:0C4CFF00740AF0D226900000E004F022BD
:1051E800302365900001E0FF900034F0C223BF2A0D
:1051F800079000007403F022900034E0FFB4230805
:10520800900000E004F0803DEF547FFF121E6F9085
:105218000034E0547FFF90003CE0FE04F074032E5D
:10522800F582E43400F583EFF0900041E02409FFB3
:10523800E433FE90003CE0D39FEE6480F8748098DD
:095248004006900000E004F02291
:1058530030234B900001E0FF900034F0C223BF2AB5
:10586300079000007403F022900034E0FFB4230B90
:10587300900000E004F0E004F08010126682500F04
:10588300900034E090003EF0900000E004F0227BB2
:0F589300FF7A0E791A1262A990000074FAF022BF
:1048C700202303024963900001E0FF900034F0C207
:1048D70023BF2A079000007403F022900034E0FF02
:1048E700B4230A900000E004F0E004F0221266828C
:1048F700505B90003EE0540F75F00AA4FF9000341F
:10490700E0540F2FF0E0900C8693FF900034F012E4
:104917001E6F900034E0FF90003CE0FE04F074034B
:104927002EF582E43400F583EFF0900041E024098E
:10493700FFE433FE90003CE0D39FEE6480F8748080
:1049470098900000E0400304F02214F0227BFF7AE5
:0D4957000E791A1262A990000074FAF02285
:106469003020099000DCE0F54D126566302203E426
:10647900F54D30210B301E05754D0A8003754D28E9
:07648900900000E004F02286
:10517E00E54D70651242B5900040E01241A151AE6E
:10518E006451B36E51B37851B38251B38C51B8960A
:10519E0051BDA051C2AA51C7B451CCBE000051CFCF
:1051AE001265B1801C126305801712681D801212E1
:1051BE00681E800D12681F80081268208003126816
:1051CE002130200F9000DEE09000A1F0900000E072
:0A51DE0004F0229000007401F0229A
:106672009000A1E070091265809000007401F02280
:1054FD0030200D9000DCE0F54D126566E54D70FC39
:10550D00302107754D05E54D70FCE4F54F30210C4C
:10551D001266CE1224C21267281224C230200C1239
:10552D0066D91224C21267281224C2054FE54FC353
:10553D00940540D930200E9000DEE09000A1F0904F
:0C554D0000A1E070FA9000007401F02250
:01681900225C
:01681A00225B
:01681B00225A
:104C120030210A201E079000007401F02230200D7E
:104C22009000DCE0F54D126566E54D70FC30210721
:104C3200754D05E54D70FC30201B9000BFE0F52A54
:104C42001266D9E4F54F1224C2054FE54FC3940A08
:104C520040F412672830211B9000C0E0F52A12664A
:104C6200CEE4F54F1224C2054FE54FC3940A40F437
:104C720012672830200E9000DEE09000A1F0900034
:0D4C8200A1E070FA121ED6E4900000F022AE
:01681C002259
:105DB10030133E20233B9000A47464F0E542547FED
:105DC100FF900A7D93900001F030260EE54230E706
:105DD10009EF900A8D93900001F0D223C213900035
:105DE10001E0B42307900002E004F022E4900002F5
:025DF100F0229E
:105DF30030113E20233B9000A47464F0E540547FAF
:105E0300FF900A7D93900001F030260EE54030E7C5
:105E130009EF900A8D93900001F0D223C2119000F4
:105E230001E0B42307900002E004F022E4900002B2
:025E3300F0225B
:10287F00202403022A31302303022A31900002E080
:10288F00F552E4F09000A47464F01268108F51D2E6
:10289F0023E551B430079000017430F022E551B4B4
:1028AF0031079000017431F022E551B432079000E6
:1028BF00017432F022E551B433079000017433F004
:1028CF0022E551B434079000017434F022E551B47D
:1028DF0035079000017435F022E551B436079000AA
:1028EF00017436F022E551B437079000017437F0C8
:1028FF0022E551B438079000017438F022E551B445
:10290F0039079000017439F022E551B4231090007B
:10291F00017423F0AF520552900002EFF022E551FF
:10292F00B42A07900001742AF022E551B4410790B0
:10293F0000017441F022E551B44207900001744246
:10294F00F022E551B443079000017443F022E551A2
:10295F00B464079000017444F022202603C223229E
:10296F00E551B461079000017461F022E551B46242
:10297F00079000017462F022E551B46307900001E3
:10298F007463F022E551B464079000017464F0227F
:10299F00E551B465079000017465F022E551B46606
:1029AF00079000017466F022E551B46707900001AB
:1029BF007467F022E551B468079000017468F02243
:1029CF00E551B469079000017469F022E551B46ACA
:1029DF0007900001746AF022E551B46B0790000173
:1029EF00746BF022E551B46C07900001746CF02207
:1029FF00E551B46D07900001746DF022E551B46E8E
:102A0F0007900001746EF022E551B46F079000013A
:102A1F00746FF022E551B470079000017470F022CA
:032A2F00C223229D
:0B669E007F209000037420F0A3DFFCBD
:0166A90022CE
:0F668200EFC394304007EFD39439500122C32265
:104DF90090000CE0FD6420602E90000BE0540F75CC
:104E0900F00AA4FBAAF090000AE0540F75F064A41C
:104E19002BFFE5F03AFEED540F7C002FFFEC3E909E
:104E29000071F0A3EF803190000BE0FD6420900049
:104E39000A601AE0540F75F00AA4FFED540F7C00C4
:104E49002FFEEC35F0900071F0A3CE800BE0540FEB
:104E5900FF900071E4F0A3EFF0E024FFF0900071FF
:054E6900E034FFF0221F
:1052B900900009E0FD6420602B900008E0540F7510
:1052C900F00AA4FBAAF0900007E0540F75F064A45B
:1052D9002BFFE5F03AFEED540F7C002FFFEC3E90DA
:1052E9000073802E900008E0FD6420900007601A8A
:1052F900E0540F75F00AA4FFED540F7C002FFEEC6B
:1053090035F0900073F0A3CEF022E0540FFF900027
:0753190073E4F0A3EFF022A2
:10652600900005E0540F75F00AA4FFA3E0540F2F66
:10653600900035F0D394004006E09415500122C334
:016546002232
:1054A000E4FFEF75F003A4249DF582E4340AF5834C
:1054B000E493FE900004E0FDEE6D703BEF75F003A9
:1054C000A4249EF582E4340AF583E493FE9000055B
:1054D000E0FDEEB50521EF75F003A4249FF582E40D
:1054E000340AF583E493FE900006E0FDEEB505076F
:0C54F000900036EFF0D3220FBF33A7C3AB
:0154FC00228D
:1053E200E4FF75F003EFA42436F582E5F0340BF503
:1053F20083E493FE900004E0FDEE6D703D75F003D2
:10540200EFA42437F582E5F0340BF583E493FE90A4
:105412000005E0FDEEB5052275F003EFA42438F592
:1054220082E5F0340BF583E493FE900006E0FDEE96
:0F543200B50507900037EFF0D3220FBF70A4C36A
:015441002248
:1041C70074032FF582E43400F583E0FD64317069F0
:1041D700FE74042FF582E43400F583E0FCEE75F0FD
:1041E70003A4249DF582E4340AF583E4936C7042BA
:1041F70074052FF582E43400F583E0FCEE75F003D7
:10420700A4249EF582E4340AF583E493B504237469
:10421700062FF582E43400F583E0FCEE75F003A485
:10422700249FF582E4340AF583E493B50404EE048D
:10423700FF220EBE339B7F0022ED6432706DFE7449
:10424700042FF582E43400F583E0FD75F003EEA456
:104257002436F582E5F0340BF583E4936D704574ED
:10426700052FF582E43400F583E0FD75F003EEA435
:104277002437F582E5F0340BF583E493B50525740F
:10428700062FF582E43400F583E0FD75F003EEA414
:104297002438F582E5F0340BF583E493B50505EE94
:0D42A7002434FF220EBE70977F00227F009E
:0142B40022E7
:104A9200EFC3943390006C50397431F0EF75F0032A
:104AA200A4249DF582E4340AF583E49390006DF02A
:104AB200EF75F003A4249EF582E4340AF583E493AF
:104AC20090006EF0EF75F003A4249FF582E4340A9F
:104AD200803A7432F075F003EFA4249DF582E5F07C
:104AE200340AF583E49390006DF075F003EFA4248B
:104AF2009EF582E5F0340AF583E49390006EF0753A
:104B0200F003EFA4249FF582E5F0340AF583E493E1
:054B120090006FF0228D
:1065C800900005E0540F75F00AA4FFA3E0540F2FC4
:0565D800900038F022E4
:1065DD00900005E0540F75F00AA4FFA3E0540F2FAF
:0565ED00900039F022CE
:1065F200900005E0540F75F00AA4FFA3E0540F2F9A
:0566020090003AF022B7
:1065030090004BE0FF90004AE08FF0A4FF90004919
:10651300E07C002FFFEC35F0FE900042E02FFFEC13
:036523003EFE2217
:10660700900044E075F010A4244DF9740235F0FAB7
:056617007BFF0262DAC6
:036810007F0322E1
:1065B100302008900023E0FF1266B63021089000D9
:0765C10023E0FF1266AA228D
:10630500E4F55E900033E0FFE55EC39F5021742302
:10631500255EF582E43400F583E0F55F302004FF67
:0F6325001266B6302105AF5F1266AA055E80D4FE
:016334002246
:01681D002258
:01681E002257
:01681F002256
:016820002255
:016821002254
:0C66AA001266E41224C212672F0224C200
:0C66B6001266EF1224C212672F0224C2E9
:1042B500E4F55EF55FF560900072E02401FF900083
:1042C50071E03400FEC3EF940AEE94005005A3E0BC
:1042D50004F560D3EF9463EE9400404C900072E0D7
:1042E5002401FB900071E03400FA7C007D64AF038B
:1042F500FE12412A8F5EEF75F064A4FFC3EB9FFFAA
:10430500EA95F0FE7C007D0A12412A8F5FA3E00446
:10431500FFE55E75F064A4FEC3EF9EFFE55F75F0F3
:104325000AA4FEC3EF9EF560900072E02401FF90A1
:104335000071E03400FED3EF9409EE940040197C3F
:10434500007D0A12412A8F5FA3E004FFE55F75F047
:104355000AA4FEC3EF9EF5607430255EF55E7430E9
:10436500255FF55F74302560F560302014AF5E126F
:1043750066B6AF5F1266B6AF601266B67F2A126682
:10438500B6302114AF5E1266AAAF5F1266AAAF609F
:084395001266AA7F2A1266AA33
:01439D0022FD
:0662A3007BFF7A0D798AF1
:0662A9008B5F8A60896131
:1062AF007F01121E9EE4F562AB5FAA60A961856251
:1062BF00827583001240EBFF121E6F0562E562C309
:0462CF00941040E403
:0162D30022A8
:0662D4007BFF7A0D79DA70
:0662DA008B608A618962FD
:1062E0007F11121E9EE4F563AB60AA61A96285630B
:1062F000827583001240EBFF121E6F0563E563C3D6
:04630000941040E4D1
:016304002276
:105EB3007BFF7A0E794A1262DA12601BE4F55EF513
:105EC3005FE55F900A3C93FDAF5FAE5E124964E508
:105ED3005F900A3C93FDAF5FAE5E125AF9055FE532
:0E5EE3005F7002055EC3943AE55E940040D302
:015EF100228E
:016822002253
:016823002252
:016824002251
:016825002250
:01682600224F
:01682700224E
:01682800224D
:106490007BFF7A0E79CA1262A9125EB312682212C9
:1064A0006823126824126825126826126827126869
:0764B00028121EB8021EC7EE
:10633500755E01755F007560B3E4F561AF617E0060
:106345001249A5AB5E0560E560AA5F7002055F14A2
:0E635500F9EF1241180561E561C3943A40DE8C
:016363002217
:1064180012601BE4F55EF55FAF5FAE5E1249A5AD95
:1064280007AF5FAE5E125AF9055FE55F7002055E61
:09643800C3943AE55E940040DFD4
:016441002238
:1064B700E4F564F565AF65AE64126392AD07AF6549
:1064C700AE641249640565E56570020564C3943AD4
:0664D700E564940040DFC3
:0164DD00229C
:10608E00755E01755F007560B3E4F561F562AF6230
:10609E00AE61126392AB5E0560E560AA5F700205A9
:1060AE005F14F9EF1241180562E56270020561C3D3
:0860BE00943AE561940040D61C
:0160C60022B7
:1060C700755E01755F007560B3E4F561F562AB5EFF
:1060D7000560E560AA5F7002055F14F91240D2FD02
:1060E700AF62AE611249640562E56270020561C381
:0860F700943AE561940040D6E3
:0160FF00227E
:10496400C2B0758400D2C2C2C6D2C6C2C4D2C5C245
:10497400C330C3FD74A0F5C2C2C5C2C330C3FD8E2B
:10498400C2C2C330C3FD8FC2C2C330C3FD8DC2C215
:10499400C330C3FDD2C4C2C320C4FD1224AAD2B002
:1049A40022758400C2C3D2C530C3FD74A0F5C2C24F
:1049B400C5C2C330C3FD8EC2C2C330C3FD8FC2C2E1
:1049C400C330C3FDC2C4D2C5C2C330C3FD74A1F594
:1049D400C2C2C5C2C330C3FDC2C2C2C330C3FD8597
:1049E400C207D2C4C2C320C4FD22D2C2C2C6D2C628
:0849F400D2C4C2C320C4FD229D
:102D8300754700122D9E50FB22754700122E2750C7
:102D9300FB22754700122DDE50FB22758400E547A8
:102DA30075F003A4902DAB73022E43022E52022E14
:102DB30070022E59022E7C022E83022E8B022E527B
:102DC300022E99022E59022EA9022EB2022E43027E
:102DD3002E52022EC0022E59022ECC758400E547D6
:102DE30075F003A4902DEB73022E43022E52022E94
:102DF30070022E59022E7C022E83022E43022E5283
:102E0300022E70022E59022E7C022E83022E7C0289
:102E13002E83022E8B022E52022ECE022E59022E0A
:102E2300A9022ECC758400E54775F003A4902E34D7
:102E330073022E43022E52022EC0022E59022ECCB2
:102E4300C2FA122EDE122EDE759B000547C3223016
:102E5300F9020547C32230F912E59A20E7FB122E47
:102E6300DED2FA122EDE122EDE0547C322C2FA127A
:102E73002EDE759B040547C322753A1E0547C32200
:102E8300E53A70020547C322C2FA122EDE122EFF64
:102E9300F59B0547C322C2FA122EDE122F0E4407FA
:102EA300F59B0547C322122EF0F53B0547C3227558
:102EB300840F30DE04E53B70020547C322C2FA12D9
:102EC3002EDE759B080547C322D322C2FA122EDEDB
:092ED300122F0E4405F59B054782
:102EDC00C322000000000000000000000000000001
:102EEC0000000022902EF7E54893225A5A5A5A5A5B
:102EFC00FAFAFA902F06E548932200B45AE12D878E
:102F0C007ADB902F15E5489322000000000000802A
:012F1C008034
:105D2A002A2A3132333435362A2A2A2A313233346E
:105D3A0035302A2A44313233343536373839302A25
:105D4A0023414243202056455253494F4E20322E7A
:105D5A0031312020202020205349454D454E5320E3
:045D6A0020202020B5
:10481B00302920C229E542540F905D3E9390008CC5
:10482B00F0786876329000B4E060151261A1125FE7
:10483B00A5800D7868E67008900078F0900089F0FC
:10484B00302A40C22AE540540F905D3E9390008B76
:10485B00F0754A32125B42301E06740044B3700985
:10486B00201E099000B5E06003125F6A301E0674CB
:10487B000044B37003201E0312616C201E151262DC
:10488B003F8010E54A700C900079F0900088F09012
:10489B0000EDF03025199000B6E0601F754B321219
:1048AB00681390007CEFF0C225125FE00261D6E541
:0C48BB004B700890007AF090008AF02208
:10616C00900079E0FF04F0EF905D2A93FF90008B94
:10617C00E0FEEF6E6011EEB42A089000797401F025
:10618C008005E4900079F0900079E0B40A06E4F020
:05619C00D221D22B22EC
:1061A100900078E0FF04F0EF905D2A93FF90008C5F
:1061B100E0FEEF6E6011EEB42A089000787401F0F1
:1061C1008005E4900078F0900078E0B40A06E4F0ED
:0561D100D220D22B22B8
:1061D60090007AE0FF04F0EF905D2A93FF90007C38
:1061E600E0FEEF6E6011EEB42A0890007A7401F0BA
:1061F6008005E490007AF090007AE0B40A06E4F0B4
:05620600D222D22B2280
:105F6A00900088E0FF04F0747F2FF582E43400F596
:105F7A0083E0FF90008BE0FEEF6E6011EEB4230821
:105F8A009000887401F08005E4900088F090008801
:0B5F9A00E0B40906E4F0D221D21F227F
:105FA500900089E0FF04F0747F2FF582E43400F55A
:105FB50083E0FF90008CE0FEEF6E6011EEB42308E5
:105FC5009000897401F08005E4900089F0900089C3
:0B5FD500E0B40906E4F0D220D21F2245
:105FE00090008AE0FF04F0747F2FF582E43400F51E
:105FF00083E0FF90007CE0FEEF6E6011EEB42308BA
:1060000090008A7401F08005E490008AF090008A84
:0B601000E0B40906E4F0D222D21F2207
:10623F0090007BE0FF04F0EF905D3493FF90008BB4
:10624F00E0FEEF6E6011EEB42A0890007B7401F04F
:10625F008005E490007BF090007BE0B40A04E4F04A
:03626F00D22C220C
:1063C00090007F7423F0A3F0E4FF74B72FF582E40C
:1063D0003400F583E0FE74812FF582E43400F58308
:0C63E000EEF00FBF06E49000877423F07D
:0163EC00228E
:10580300121DCC121EB87F01121E9E7BFF7A5D799A
:105813005E1262A97BFF7A5D794E1262DA753914E2
:10582300E490007EF090007DF0FF744C2FF582E44D
:105833003400F583E4F0745C2FF582E43400F583DF
:10584300E4F00FBF10E4E53970FC121EB8021EC766
:104FC40090007EE0FFD3940F501FEF04FF121E9E4B
:104FD40090008BE0FF90007EE0FE04F0744C2EF510
:104FE40082E43400F583EF80437F01121E9EE4F5D2
:104FF4005E744D255EF582E43400F583E0FF744C65
:10500400255EF582E43400F583EFF0744C255EF5FB
:1050140082E43400F583E0FF121E6F055EE55EC393
:10502400940F40CD90008BE0FF90005BF0121E6F58
:015034002259
:104EE10090007DE0FFD3940F5020EF2411FF121E9C
:104EF1009E90008CE0FF90007DE0FE04F0745C2E3B
:104F0100F582E43400F583EF80437F11121E9EE4A5
:104F1100F55E745D255EF582E43400F583E0FF748F
:104F21005C255EF582E43400F583EFF0745C255E68
:104F3100F582E43400F583E0FF121E6F055EE55E45
:104F4100C3940F40CD90008CE0FF90006BF0121ED7
:014F51006FF0
:014F5200223C
:036813007F0122E0
:105B42009000EDE0FF700E90008BE0B42A07900009
:105B5200ED7401F022EFB4011390008BE0B423073F
:105B62009000ED7402F022E49000EDF09000EDE080
:105B7200B4021490008BE0B430089000EE7401F08F
:085B82008000E49000EDF02228
:10439E00E53760021537E53A6002153A900093E072
:1043AE00600214F0900097E0600214F090009BE021
:1043BE00600214F090009FE0600214F09000A2E002
:1043CE00600214F09000AAE0600214F09000B2E0D7
:1043DE00600214F022E538600215389000A1E0600A
:1043EE000214F0900092E0600214F0900096E060EB
:1043FE000214F09000A7E0600214F022E53960028A
:10440E001539E53B6002153BE54C6002154CE54D58
:10441E006002154D7868E6600116E54A6002154A9D
:10442E00E54B6002154B9000AFE0600214F0900077
:10443E009AE0600214F090009EE0600214F090008A
:10444E00A8E0600214F09000EFE0600214F0222267
:10445E009000A4E0600214F0229000A3E060021429
:02446E00F0223A
:10201600202046554E4354494F4E2031382020202B
:1020260000202020454D455247454E43592020204B
:102036002000202020205354414E44425920202085
:102046002020524144494F204F524947494E41545E
:10205600452054454C434F204F524947494E415421
:10206600452020202046554E4354494F4E203120CE
:10207600202020202046554E4354494F4E203220E2
:10208600202020202046554E4354494F4E203320D1
:10209600202020202046554E4354494F4E203420C0
:1020A600202020202046554E4354494F4E203520AF
:1020B600202020202046554E4354494F4E2036209E
:1020C600202020202046554E4354494F4E2037208D
:1020D600202020202046554E4354494F4E2038207C
:1020E600202020202046554E4354494F4E2039206B
:1020F6002020202052454345495645204D4F444512
:102106002020205452414E534D4954204D4F4445B2
:102116002020202046554E4354494F4E2031302032
:102126002020202046554E4354494F4E2031312021
:102136002020202046554E4354494F4E2031322010
:102146002020202046554E4354494F4E20313320FF
:102156002020202046554E4354494F4E20313420EE
:102166002020202046554E4354494F4E20313520DD
:102176002020202046554E4354494F4E20313620CC
:102186002020202046554E4354494F4E20313720BB
:102196002020202046554E4354494F4E20313820AA
:1021A6002020202046554E4354494F4E2031392099
:1021B6002020202046554E4354494F4E2032302091
:1021C6002020202046554E4354494F4E2032312080
:1021D6002020202046554E4354494F4E203232206F
:1021E6002020202046554E4354494F4E203233205E
:1021F6002020202046554E4354494F4E203234204D
:102206002020202046554E4354494F4E203235203B
:102216002020202046554E4354494F4E203236202A
:102226002020202046554E4354494F4E2032372019
:1022360020203A0036AA340031552EAA2C00295502
:0E22460026AB240021551EAB1C0019551400B8
:101B75009000E8E07003021DCB202D0F9000B0E02F
:101B850060099000AFE07003021DC7202D03021D00
:101B9500CBC22D9000B0E0FF7027E540B40B0C9050
:101BA50000AF7414F09000B0E004F0E540640C6000
:101BB50003021DCB9000AF7414F09000B07403F0D5
:101BC50022EF64016003021CD2E540B40B03021D41
:101BD50075E540B40C0D9000AF7414F09000B0742E
:101BE50004F0229000DBE0C39403502EE5409400FE
:101BF5004028E54094085022E540149000ACF09050
:101C050000AE7401F09000ACE075F010A42468F902
:101C1500742035F0FA7BFF1262A99000DBE0B40373
:101C25002FE540D394074028E540940A5022E5402B
:101C3500149000ACF09000AE7401F09000ACE0752B
:101C4500F010A42468F9742035F0FA7BFF1262A91C
:101C55009000DBE064047035E5406408702F7BFF7D
:101C65007A2079D81262A97BFF7A2179081262DA83
:101C75009000EBE0B403031267369000ECE0B40388
:101C8500031267421265669000B17401F09000DBA3
:101C9500E064047034E5406409702E7BFF7A207996
:101CA500E81262A97BFF7A2079F81262DA9000EBDC
:101CB500E0B4030312673C9000ECE0B40303126741
:101CC50048126580E49000B1F0E4021DC79000B0B1
:101CD500E064036003021D68E540B40C03021D7552
:101CE500E540B40B03021D81E540B4092E9000AC1C
:101CF500E09000ADF09000AC7414F0E49000ABF00F
:101D05009000AE04F07BFF7A2079161262A97BFF62
:101D15007A2079271262DAE4021DC79000DBE0C35E
:101D250094035007E540C394084005E540B40A30E4
:101D3500E540B40A089000AC7409F08008E5402439
:101D4500099000ACF09000AE7401F09000ACE07525
:101D5500F010A42488F9742035F0FA7BFF1262A9EB
:101D6500E4805F9000B0E06404705BE540B40C076C
:101D75009000AF7414F022E540B40B0D9000AF74E1
:101D850014F09000B07401F0229000DBE0C39403DE
:101D9500502FE54094004029E540940A5023E54042
:101DA50024149000ACF09000AE7401F09000ACE00B
:101DB50075F010A42458F9742035F0FA7BFF1262EF
:071DC500A9E49000B0F02238
:1017D5009000DBE064047003021B749000AEE070BF
:1017E50003021B741267DA9000ABE0FF70309000C3
:1017F500ACE0FE64076011EEC39405400BEED39494
:1018050013400CEE941850079000AB7401F022EED3
:101815009000ABB408047408F0227404F022EFB40D
:1018250001030219599000ABE0640260030218E05D
:101835009000AAE06003021B749000ACE0FF600317
:10184500B4070C90223CE493F516740193F517EF59
:10185500B4010C90223EE493F516740193F517EF4D
:10186500B4020C902248E493F516740193F517EF32
:10187500B4030C90224AE493F516740193F517EF1F
:10188500B4040C902244E493F516740193F517EF14
:10189500B4140C90223AE493F516740193F517EFFE
:1018A500B4150C902246E493F516740193F517EFE1
:1018B500B4160C902240E493F516740193F517EFD6
:1018C500B4170C902242E493F516740193F5179022
:1018D50000C4E0F5281267E0021A569000ABE064F8
:1018E50003706A9000AAE06003021B74902238938B
:1018F500F516740193F5179000C5E0F5281267E019
:101905009000B17401F01267BCE49000ABF0900058
:10191500AEF09000ACE064146003021B749000AD5F
:10192500E09000ACF01267E3121EB8E49000B1F04D
:1019350090009CF0900099F09000DEE0FF9000D9B7
:10194500E02F9000A1F09000A5740AF0229000AB62
:10195500E0B40420902238E493F516740193F5174A
:101965009000C6E0F5281267E01267DA9000AA74C5
:1019750078021B269000ABE0FF64056003021A5E47
:101985009000AAE06003021B749000ACE0FEB40571
:101995000C90224CE493F516740193F517EEB406FA
:1019A5000C90224EE493F516740193F517EE640935
:1019B5006004EEB4180C90224CE493F51674019370
:1019C500F517EE640A6004EEB4190C90224CE4930A
:1019D500F516740193F517EE640B6004EEB41A0C5A
:1019E50090224CE493F516740193F517EEB40C0CA4
:1019F50090224CE493F516740193F517EEB40D0C93
:101A050090224EE493F516740193F517EE640E607B
:101A150004EEB41B0C90224EE493F516740193F575
:101A250017EE640F6004EEB41C0C90224EE493F59F
:101A350016740193F517EE64106004EEB41D0C9056
:101A4500224EE493F516740193F5179000C4E0F562
:101A5500289000AA7428021B26EF64066003021B67
:101A65002E9000AAE06003021B749000ACE0FF64B6
:101A7500056004EFB4060C90223CE493F51674015E
:101A850093F517EF64096004EFB40D0C90223EE462
:101A950093F516740193F517EF640A6004EFB40E1D
:101AA5000C902248E493F516740193F517EF640B37
:101AB5006004EFB40F0C90224AE493F51674019379
:101AC500F517EF640C6004EFB4100C902244E49316
:101AD500F516740193F517EF64186004EFB41B0C49
:101AE500902246E493F516740193F517EF64196097
:101AF50004EFB41C0C902240E493F516740193F5A1
:101B050017EF641A6004EFB41D0C902242E493F5BC
:101B150016740193F5179000C4E0F5289000AA7497
:101B250028F09000ABE004F0229000ABE0FFB40792
:101B3500279000AAE0703890223893F51674019327
:101B4500F5179000C5E0F5289000B17401F0E49018
:101B550000ABF09000AEF022EFB408131267E31269
:101B650067DDE49000ABF09000AEF09000B1F0229C
:10247E00000000000000000000000000000022C06C
:10248E0000C001790478B4D8FED9FAD001D0002268
:10249E00C000781412248DD8FBD00022C0E075370E
:1024AE0005E53770FCD0E022C0E075370FE53770D8
:1024BE00FCD0E022C0E0753764E53770FCD0E02236
:1024CE00A42582F582E58335F0F58322B40A002235
:1024DE00C0E0C3997001D3D0E022B50601225007A7
:1024EE00B5070122400122D322EF75F06484243017
:1024FE0090006CF0E5F0A375F00A842430F0A3E5AB
:10250E00F02430F022EF75F06484243090006CF0EB
:10251E00E5F0A375F00A842430F0A3E5F02430F042
:10252E0090006CE0B4300B7420F0A3E0B430037470
:10253E0020F02290000DE0540FFFA3E0B4200280A3
:10254E0019540FCF75F00AA42FFFA3E0B420028018
:10255E0009540FCF75F00AA42FFF22C006C005C084
:08256E000490000DE0540FFF82
:10257600FEA3E0B42003C3802C540FFDCF75F00AF0
:10258600A42FFFA3E0B42003C3801A540FFCEE75FA
:10259600F064A420D20EFEED75F00AA42E40052CA0
:1025A60040028001D3D004D005D0062275F06484A1
:1025B600F6E5F00875F00A84F608A6F00822C001D0
:1025C6007900E6B4FF028027F908E6B4FF03C3806A
:1025D60022E975F00AA426F908E6B4FF03C38013BE
:1025E600E975F00AA420D207C3264003F98004D374
:1025F600D00122E9D00122E675F00AA40826227845
:1026060047EE1225B2754500754600784990265E5C
:102616007908EF134007A3A3A3A3A3801CC0E0C0BF
:1026260000C001C37905E49336D4A2E4540FF6A39F
:1026360018D9F3D001D000D0E0D9D8E545600C75A3
:102646004609754709754809754909854645854707
:1026560046854847854948220605020000020105CD
:10266600000004020001000804000200060900043C
:102676000002090108000408030601080607020310
:1022540020205455524E204F4E20535720202020EA
:102264000020205455524E204F46462053572020DC
:10227400200044313233343536373839302A23415B
:10228400424302AB055508000AAB0D55100012ABD2
:10229400155518001AAB1D55200022AB25552800F2
:1022A4002AAB2D55300032AA3555202054455354BD
:1022B40020524F5554494E45202020205645525314
:1022C400494F4E20312E302020202054455354496C
:1022D4004E4720454550524F4D20202054455354DD
:1022E400494E4720564F49434520205445535449AD
:1022F4004E472044544D46203120205445535449E0
:102304004E472044544D46203220202054455354F7
:10231400494E4720525332333220202054455354DF
:10232400494E4720525334383520202020544553F9
:1023340054494E472050545420202054455354208F
:102344004155582052454C4159202054455354205E
:1023540043542052454C4159202020544553494E62
:10236400472052494E47494E472020202020202014
:102374002020202020202020202020544553542099
:102384004C494E452052414C415954455354204CDC
:10239400494E452053454E53452B54455354204CE8
:1023A400494E452053454E53452D20205445535402
:1023B400204449475F494E2020202054455354204F
:1023C400494E50555420564F4C5420544553542094
:1023D4004C494E452052454C415954455354205A7A
:1023E40045524F2043524F53532054455354494E62
:1023F4004720535155454C434820202054455354BD
:10240400494E47204850462020202054455354200C
:1024140054454C434F20564F582020544553542084
:10242400524144494F20564F58202054455354207C
:10243400454D5F4F50545020202020202020202044
:102444002020202020202020202020202020202088
:1024540020202020202020202020205445535420B8
:10246400434F4D504C45544544202020205445535F
:0A24740054204641494C4544202005
:100EDA007BFF7A2279AE1262A97BFF7A2279BE124F
:100EEA0062DA1267107BFF7A2279CE1262A9121E89
:100EFA00C71267107F007E001249A58F4F7DAA7F17
:100F0A00007E001249647F007E001249A5EF64AAA0
:100F1A00600C7BFF7A24796E1262DA1268167D55AC
:100F2A007F007E001249647F007E001249A5EF64AB
:100F3A0055600C7BFF7A24796E1262DA126816AD5C
:100F4A004F7F007E001249647BFF7A24795E126229
:100F5A00A91267107BFF7A2279DE1262A9126754FE
:100F6A001266CE754700754801753914122D95E53C
:100F7A003970FC122D8C12679075470075480175FF
:100F8A003905E53970FCD202D20A122D83C202C297
:100F9A000A7BFF7A24795E1262A91267107BFF7AB4
:100FAA002279EE1262A9121EC71267107F311266E9
:100FBA00EF753932E53970FC12672F3013FD12676D
:100FCA002FE542547FFFEF90227693FFEFB4310E64
:100FDA007BFF7A24795E1262A9126710800C7BFF6C
:100FEA007A24796E1262DA1268167BFF7A2279FE07
:100FFA001262A9121EC71267107F311266E41267C5
:10100A001812672F3011FDE540547FFFEF902276CA
:10101A0093FFEFB4310E7BFF7A24795E1262A91234
:10102A006710800C7BFF7A24796E1262DA126816D6
:10103A007BFF7A23790E1262A9121EC712671075F6
:10104A008400759850C299C2987599433098FD7575
:10105A008400E5996443600C7BFF7A24796E1262FE
:10106A00DA1268167BFF7A24795E1262A912671077
:10107A007BFF7A23791E1262A9121EC71267101209
:10108A006798758400759850C299C29875994330CB
:10109A0099FD7BFF7A24795E1262A91267107BFFA1
:1010AA007A23792E1262A9121EC712671012656678
:1010BA00126718E53ED39432400C7BFF7A24796E8E
:1010CA001262DA126816126580126718E53EC39436
:1010DA00AA500C7BFF7A24796E1262DA1268167BA8
:1010EA00FF7A24795E1262A91267107BFF7A23794C
:1010FA003E1262A9121EC7126710126736126718CB
:10110A00E53DD3940A400C7BFF7A24796E1262DAA9
:10111A0012681612673C126718E53DC394AA500C70
:10112A007BFF7A24796E1262DA1268167BFF7A24C0
:10113A00795E1262A91267107BFF7A23794E1262D6
:10114A00A9121EC71267101267421267101267109F
:10115A001267487BFF7A24795E1262A91267107BB4
:10116A00FF7A23797E1262A9121EC71267101267CC
:10117A004E12671012671012675412671012671026
:10118A007BFF7A2379AE1262A9121EC7126710304A
:10119A00DC1D7BFF7A2279541262DA20DCFD121EF2
:1011AA00C77BFF7A24795E1262A9126710801B7BC3
:1011BA00FF7A2279651262DA30DCFD121EC77BFFE4
:1011CA007A24795E1262A91267107BFF7A24792E3B
:1011DA001262A9121EC7126710126778501F7BFF8E
:1011EA007A2279541262DA12677840FB121EC77BA0
:1011FA00FF7A24795E1262A9126710801D7BFF7A3A
:10120A002279651262DA12677850FB121EC77BFFD9
:10121A007A24795E1262A91267107BFF7A2379BE5B
:10122A001262A9121EC7126710E53CC3940A40074E
:10123A00E53CD39446400C7BFF7A24796E1262DA3D
:10124A001268167BFF7A24795E1262A91267107BF4
:10125A00FF7A2379DE1262A9121EC712671012667C
:10126A00FA1267B340FB1267B350FB1267B340FB35
:10127A007BFF7A24795E1262A91267101267287BB3
:10128A00FF7A2379EE1262A9121EC712671012673B
:10129A005A400F12656612658012675A50F580022D
:1012AA0080F17BFF7A24795E1262A91267107BFFB4
:1012BA007A24791E1262A9121EC7126710126705D4
:1012CA0012676050FB800280F71267287BFF7A243E
:1012DA00795E1262A91267107BFF7A2379FE126285
:1012EA00A9121EC71267101266FA12672090228886
:1012FA00E493F508740193F50912672090228AE4B1
:10130A0093F508740193F50912672090228CE493EF
:10131A00F508740193F50912672090228EE493F57B
:10132A0008740193F509126720902290E493F50856
:10133A00740193F509126720902292E493F50874D8
:10134A000193F509126720902294E493F508740139
:10135A0093F509126720902296E493F50874019395
:10136A00F509126720902298E493F508740193F521
:10137A000912672090229AE493F508740193F509FB
:10138A0012672090229CE493F508740193F50912E0
:10139A00672090229EE493F508740193F509126779
:1013AA00209022A0E493F508740193F509126720AE
:1013BA009022A2E493F508740193F509126720902C
:1013CA0022A4E493F508740193F509126720902288
:1013DA00A6E493F508740193F5091267209022A8F0
:1013EA00E493F508740193F5091267209022AAE4A0
:1013FA0093F508740193F5091267209022ACE493DF
:10140A00F508740193F5091267287BFF7A24795E3F
:09141A001262A91267100212F11E
:0114230022A6
:0867100075390AE53970FC221D
:08671800753902E53970FC221D
:08672000753905E53970FC2212
:0368160080FE22DF
:08000300022A32000000000097
:08000B00022A3300000000008E
:08001300022B66000000000052
:08001B003200000000000000AB
:09002300320000000000000000A2
:08002B00022A3600000000006B
:08003300320000000000000093
:0A003B003200000000000000000089
:0900430032000000000000000082
:08004B0032000000000000007B
:08005300320000000000000073
:08005B00022A980000000000D9
:08006300320000000000000063
:08006B00022AB70000000000AA
:08007300022A3C00000000001D
:08007B00022B670000000000E9
:08008300022A950000000000B4
:08008B0032000000000000003B
:10009300022B8500000000000000000000000000AB
:1000A3003275FF0775FFDE75FFAD75840F75E107C8
:1000B30075E20475E34475840F75A43575A5097558
:1000C300A6FF75A7FF759CFF759D00759E00759F24
:1000D300F075D8FF75E8FF75F80F75AD0F758401DE
:1000E30075893075888F75840275893075888F7529
:1000F300840F758A80758C67780874FF0000000090
:100103000000000000000000D5E0F1D8EDE58C30E0
:10011300E7FB759701758A0043890475840075B7F9
:100123001075840F438901758D01758F01758E02DA
:100133007480D5E0FD438902E58930E4FB759702BD
:1001430075840075D10775840075BB0175BA007598
:10015300BCF075C70075C60075C5FF75C4FF75E8AB
:100163008175840275BB0475BA0075BCF175C60050
:1001730075C4FF75E88875840075D484758401752A
:10018300D484758400C2F8759A47759D1A43F8099B
:1001930075870075840075B90075A90075910075A0
:1001A300985075840175981075840075C04075C3A7
:1001B3000075CFC9758400758E0075892075880513
:1001C300758400758A00758B6F758CF4758D6F431C
:1001D300885075840075C90075CA0075CB0075CC4D
:1001E3000075CD0075840175C91875CA8075CBFB80
:1001F30075CDFB75CC80D2CA75840275C91875CAD2
:10020300A675CBAF75CDAF75CCA6D2CA7584007574
:10021300A8AF75B80075E6A475E71775F60075F70E
:10022300019000007F007E20E4F0A3DFFCDEFA757E
:0202330027FFA3
:100235007528FF7529FF752AFF752BFF752CFF752E
:080245002DFFD2B61249EE2292
:105AF900AC84A2AF922EABB1C2AF75840F53A1FE95
:105B090075B121E4F58443B701F584438F01786CBD
:105B1900768008F6EF26F618EE36F6E6FE08E6F584
:105B2900828E83EDF0E4F584538FFEF58453B7FE3E
:085B39008BB18C84A22E92AF07
:015B41002241
:10639200AD84A2AF922EACB1C2AF75B12175668049
:1063A200756700EF2567F567EE3566F566856782E6
:0D63B200F583E493FF8CB18D84A22E92AF91
:0163BF0022BB
:10601B00AF84A2AF922EAEB1C2AF786C7680087609
:10602B000075B121E4F58443B701F584758F03182E
:10603B00E6FC08E6F5828C83E4F0F58FF58453B724
:09604B00FE8EB18F84A22E92AFEB
:016054002229
:030000000266C2D3
:0C66C200787FE4F6D8FD75816D0244700D
:1040D200BB010689828A83E0225002E722BBFE02EC
:0940E200E32289828A83E493221F
:1040EB00BB010CE58229F582E5833AF583E022508A
:1040FB0006E92582F8E622BBFE06E92582F8E222D4
:0D410B00E58229F582E5833AF583E49322ED
:10411800BB010689828A83F0225002F722BBFE0186
:02412800F32280
:10412A00BC000BBE0029EF8DF084FFADF022E4CC79
:10413A00F875F008EF2FFFEE33FEEC33FCEE9DEC42
:10414A00984005FCEE9DFE0FD5F0E9E4CEFD22ED88
:10415A00F8F5F0EE8420D21CFEADF075F008EF2FD2
:10416A00FFED33FD4007985006D5F0F222C398FDC3
:05417A000FD5F0EA2260
:10417F00A3F8E0C5F025F0F0E582158270021583F3
:06418F00E0C838F0E82250
:0C419500A42582F582E5F03583F5832235
:1041A100D083D082F8E4937012740193700DA3A3AD
:1041B10093F8740193F5828883E4737402936860C1
:0641C100EFA3A3A380DFC1
:00000001FF
